:020000040800F2
:1000000068660020B9020008497500088D5F000885
:100010004575000885220008ED7F000800000000FB
:100020000000000000000000000000004778000809
:1000300089220008000000004B750008C57A0008FE
:10004000D3020008D3020008D3020008D30200083C
:10005000D3020008D30200088B220008D302000854
:10006000D3020008D3020008D3020008D30200081C
:10007000D3020008D3020008D3020008D30200080C
:10008000D3020008D3020008D30200089D7F0008B5
:10009000AD7F0008D3020008D3020008D302000895
:1000A000D3020008D3020008D3020008D3020008DC
:1000B000D3020008417B0008D3020008D3020008E5
:1000C000D3020008D3020008D3020008D3020008BC
:1000D000D30200085D7F0008D3020008D3020008A5
:1000E000D3020008D3020008D3020008D30200089C
:1000F000D3020008D3020008D3020008D30200088C
:10010000D3020008D3020008D3020008D30200087B
:10011000D3020008D3020008D3020008D30200086B
:10012000D3020008D3020008D3020008D30200085B
:1001300000F002F800F0B0F80AA090E8000C824449
:100140008344AAF10107DA4501D100F0A5F8AFF226
:10015000090EBAE80F0013F0010F18BFFB1A43F0A5
:1001600001031847E09C0000009D00000A444FF086
:10017000000C10F8013B13F0070408BF10F8014B06
:100180001D1108BF10F8015B641E05D010F8016B4B
:10019000641E01F8016BF9D113F0080F1EBF10F8AF
:1001A000014BAD1C0C1B09D16D1E58BF01F801CBD2
:1001B000FAD505E014F8016B01F8016B6D1EF9D555
:1001C0009142D6D37047000000230024002500266A
:1001D000103A28BF78C1FBD8520728BF30C148BFAA
:1001E0000B6070476E2900F0D284702900F09F8167
:1001F000662909F05985652909F05685672909F0AE
:100200005385612909F0528503681B0A28BF41F014
:100210008001692900F01081642900F00D817529A1
:1002200000F00A816F2900F0D285782900F06B81F7
:10023000E92900F06D85E42900F06A85F52900F0D0
:100240006785EF2900F0CF85F82900F06A810368FF
:10025000DB0928BF41F08001632900F0DC847329A9
:1002600000F0E184E32901F02782F32901F02C82D8
:10027000002070471FB501F0C3FA040000200021E0
:1002800009F0A2FB401C60600020002109F0B2FBD5
:10029000E0601FBD10B510BD01F08DFA1146FFF7EB
:1002A000E9FF08F0F5FA01F06FFB03B4FFF7F2FF86
:1002B00003BC07F03EFF000009488047094800479B
:1002C000FEE7FEE7FEE7FEE7FEE7FEE7FEE7FEE706
:1002D000FEE7FEE704480549054A064B7047000063
:1002E000E97A000831010008686000206866002093
:1002F00068620020686200207047B2F120030AD5CE
:10030000C2F1200320FA02F001FA03F321FA02F10C
:1003100040EA0300704721FA03F04FF000017047F4
:100320007CB51D4616460C00009001D02044401EAE
:10033000074B7B442A4669460190304600F041FC59
:1003400005461CB10020694600F04EFC28467CBDE5
:10035000BD0800000FB4044910B503AA029800F0CC
:1003600067FC10BC5DF814FB1C0000200FB41CB52A
:10037000084B06AA7B4469460090059800F021FCD2
:1003800004460020694600F02FFC20461CBC5DF8A6
:1003900014FB00007108000070B504468569006810
:1003A000C10601D5302600E02026C00707D070BD69
:1003B000D4E9012130469047206A401C20626D1E1E
:1003C000F6D570BD70B5044685690078C00707D1C1
:1003D00070BDD4E9012120209047206A401C206292
:1003E0006D1EF6D570BD70B50C460546012A05D0C8
:1003F0002878800600D5EA69002302E0012305E0A1
:100400005B1C934202D2E05C0028F9D1A869E6188F
:10041000C01AA861286A184428622846FFF7BCFF62
:1004200004E0D5E9012114F8010B9047B442F8D358
:100430002846FFF7C7FF70BD2DE9F04106460024AE
:1004400010687529314616A510D000F035FB00283C
:1004500002DA404213A507E031688A0701D512A5E8
:1004600002E0490704D511A5012401E000F02DFBAD
:1004700000210A2206F1240709E0B0FBF2FCB0FBE0
:10048000F2F302FB1C00303078541846491C002857
:10049000F3D123462A463046BDE8F04100F01EBBAA
:1004A000000000002D0000002B00000020000000D4
:1004B000F0B40D460188090502D5214C7C4402E0C8
:1004C0001F4C7C440E34002100F1240608E002F0A9
:1004D0000F071209E75D42EA03721B097754491CB2
:1004E00052EA0307F3D102780023120704D5702DD6
:1004F00006D009B1022311342246F0BC00F0EEBA56
:1005000001231034F8E770B504460D462146106803
:1005100000F0DBFA024629462046BDE87040002381
:10052000C6E7D21D22F00703D3E90023C0E7036822
:10053000126843F0200303600823C3610023B7E778
:10054000389800002DE9F05F894604464FF0000A14
:10055000DFF874B1FB44C0F820A02046E16888476A
:10056000002874D0252806D0D4E901219047206ABC
:10057000401C2062F1E700265F462046E16888477C
:100580002028054607DB312D05D2781910F8200CFC
:1005900008B10643F1E7B00701D526F00406C4F818
:1005A0001CA00027C4F818A02A2D09D0284607F05F
:1005B000B9FD38B304EB8708303DC8F8185019E08E
:1005C00059F8041B204604EB87029161E1688847D3
:1005D000012F054618D1E069002820DA26F0200610
:1005E0001DE0D8F8180000EB800005EB4000303823
:1005F000C8F818002046E1688847054607F092FDD4
:100600000028EED1012F0AD02E2D08D12046E16816
:1006100088477F1C0546022F46F02006C4DBA069F0
:10062000002803DA404246F00106A061F00701D03D
:1006300026F010066C2D0BD0682D09D04C2D39D02A
:100640006A2D35D0742D35D07A2D33D016E038E0B0
:10065000E1682F4620468847B842054609D16C2FED
:1006600026D04FF48060E16806432046884705465F
:1006700004E06C2F1AD04FF4807006430DB3A5F13F
:100680004100192802D8203546F400664A4629461A
:10069000204626604E46FFF7A5FD80B101280BD00D
:1006A000F61D26F0070000F1080956E74020E4E7B0
:1006B0008020D8E70020D6E706F104094DE7284658
:1006C00052E7206ABDE8F09FC897000070B5064663
:1006D00000F0EEF90468054630460A22002100F0D9
:1006E0008DFB2C6070BD30B505460B462A4613F8CD
:1006F000014B12F8010B08B1A042F8D01CB1002840
:1007000002D06D1CF1E7284630BD40EA010310B568
:100710009B070FD1042A0DD310C808C9121F9C4291
:10072000F8D020BA19BA884201D9012010BD4FF083
:10073000FF3010BD1AB1D30703D0521C07E00020D0
:1007400010BD10F8013B11F8014B1B1B07D110F82D
:10075000013B11F8014B1B1B01D1921EF1D1184630
:1007600010BD10B5431C02E010F8011B71B18107E8
:10077000FAD14FF0013202C88C1A8C4314EAC2112C
:10078000F9D0C01A0A0603D0C01E10BDC01A10BD91
:100790000A0401D0801E10BD0902FCD0401E10BD0D
:1007A00040EA010370B59B072ED14FF00136042AB1
:1007B0002AD308C810C99D1B9D43121F15EAC615F0
:1007C00017D0D8B2E1B2401A50EA056110D198B200
:1007D000A1B2401A50EA05410AD123F07F4024F02B
:1007E0007F41401A50EA052102D1180EA0EB146097
:1007F00070BDA342DBD018BA21BA884201D90120CA
:1008000070BD4FF0FF3070BD0AB9002070BD10F808
:10081000013B11F8014B63B1A3420AD1521E08D02B
:1008200010F8013B11F8014B1BB1A34201D1521E3C
:10083000EDD1181B70BD421E12F8013F002BFBD1F9
:1008400011F8013B002B02F8013BF9D17047032A54
:1008500040F2308010F0030C00F0158011F8013BDD
:10086000BCF1020F624498BF11F801CB00F8013BC4
:1008700038BF11F8013BA2F1040298BF00F801CB88
:1008800038BF00F8013B11F0030300F06780083A1D
:10089000C0F0088051F8043B083A51F804CBA0E8B6
:1008A0000810F5E7121D5CBF51F8043B40F8043B0B
:1008B000AFF30080D20724BF11F8013B11F801CB40
:1008C00048BF11F8012B24BF00F8013B00F801CB11
:1008D00048BF00F8012B7047431A28BF9A427FF6A1
:1008E000B6AF032A1044114440F2268010F0030FE3
:1008F0001EBF11F8013D521E00F8013D10F0030F1C
:100900007FF4F6AF11F0030300F0C382083AC0F0A1
:100910000B8051F8043D083A51F804CD40F8043DED
:1009200040F804CDFFF7F3BF121D5CBF51F8043D42
:1009300040F8043DAFF30080D20724BF11F8013D19
:1009400011F801CD48BF11F8012C24BF00F8013D7A
:1009500000F801CD48BF00F8012C704710B5203ACF
:10096000C0F00B80B1E81850203AA0E81850B1E868
:100970001850A0E81850BFF4F5AF5FEA027C24BF1E
:10098000B1E81850A0E8185044BF18C918C0BDE815
:1009900010405FEA827C24BF51F8043B40F8043BDE
:1009A00008BF7047D20728BF31F8023B48BF11F893
:1009B000012B28BF20F8023B48BF00F8012B7047ED
:1009C0004FF000020429C0F0128010F0030C00F078
:1009D0001B80CCF1040CBCF1020F18BF00F8012BF6
:1009E000A8BF20F8022BA1EB0C0100F00DB85FEAC4
:1009F000C17C24BF00F8012B00F8012B48BF00F890
:100A0000012B70474FF0000200B5134694469646FE
:100A1000203922BFA0E80C50A0E80C50B1F1200111
:100A2000BFF4F7AF090728BFA0E80C5048BF0CC0BF
:100A30005DF804EB890028BF40F8042B08BF70471D
:100A400048BF20F8022B11F0804F18BF00F8012B8F
:100A5000704710B5044610F0030F08BF11F0030FE4
:100A600040F015804FF0013E121FC0F20E8051F889
:100A7000043BA3EB0E0C2CEA030C1CEACE1C08BFB3
:100A800040F8043BF0D0A1F1040102F10402521E2F
:100A900008DB11F8013B002B00F8013BF7D11146B0
:100AA000FFF78EFF204610BD7047704770477047B4
:100AB000004870470860002009684A0501D540B227
:100AC0007047C905FCD500B2704709684A0501D5D1
:100AD000C0B27047C905FCD580B270472DE9F04718
:100AE0000D4699469246044600F12408016888069E
:100AF00004D5E06921F01001216000E00120A84246
:100B000001DD471B00E00027A1697A1902EB09000B
:100B1000081AA0612078C00602D42046FFF73CFCEA
:100B2000002608E0D4E901211AF806009047206A5F
:100B3000401C761C20624E45F4DB2078C0060AD5A6
:100B40002046FFF729FC06E0D4E901213020904738
:100B5000206A401C2062381EA7F10107F4DC07E080
:100B6000D4E9012118F805009047206A401C206252
:100B7000281EA5F10105F3DC2046FFF723FC2078B1
:100B8000000602D50220BDE8F0870120FBE71168CE
:100B90000268006A530501D508700AE0D30501D543
:100BA000088006E0130603D5C217C1E9000200E081
:100BB000086001207047000001694A1C0261087842
:100BC000704700B58FB0CDE901310021059105498D
:100BD0007944CDE9031011466846FFF7B3FC0FB026
:100BE00000BD0000E5FFFFFF0A6802F8010B0A6084
:100BF0007047D1E900239A4202D2531C0B60107057
:100C0000704710B5436913B1AFF3008001E0FFF7FF
:100C1000EAFB012010BD127800F124010A700022C5
:100C20004A700122EDE711684FF0FF32E9E700005A
:100C3000074B70B50D467B44FFF7C3FF04462846BB
:100C400000F095FD10B14FF0FF3070BD204670BD33
:100C50005F7600002DE9FF5F15468A460446DFF8FF
:100C6000AC80F8440027D8E900103E46CDE90010DA
:100C700010E03AF816106A4602A800F07CFD411C0C
:100C800007D02178890603D5E269391891420DD839
:100C90000744761C2078800602D5E069B84205DD5D
:100CA000AE42E6DB3AF816000028E2D1A069C01B8C
:100CB000A0612046FFF770FBD8E90010CDE90010D5
:100CC000002017E03AF818106A4602A800F053FD19
:100CD000B0F1FF3F81460BD000250DF1080B05E078
:100CE000D4E901211BF8050090476D1C4D45F7D351
:100CF00008F10100B0428046E4DB206A38442062FB
:100D00002046FFF75FFBBDE8FF9F0000CE9000008C
:100D10002DE9F0418046D21D22F007020025D2E9DC
:100D20000002F52915A614D0011E72F1000106DAA1
:100D30000023D0EB030063EB020211A608E0D8F811
:100D400000108B0701D50FA602E0490701D50EA6BA
:100D500001251146002408F1240704E000F0D0F832
:100D600030323A55641C50EA0102F7D12B46324624
:100D700021464046BDE8F041FFF7B0BE000000004C
:100D80002D0000002B0000002000000030B40021E6
:100D900000F1240408E002F00705D208303542EAE9
:100DA0004372DB086554491C52EA0305F3D1046819
:100DB000002310A2250707D5A40600D421B1C469D9
:100DC00001230DA2641EC46130BCFFF787BE10B5BD
:100DD000044621461068FFF778FE02462046BDE82B
:100DE00010400023D2E7D21D22F00701D1E90023F1
:100DF000CCE7000000000000300000002DE9F047C3
:100E000091460F4680460446002614F8015B2DB13A
:100E100000F06EF80068405DC007F6D12B2D02D0BF
:100E20002D2D18D0641E4A463946204600F050FC4D
:100E300027B13968A14201D1C7F800804FF0020400
:100E400071050BD54042002803DDFFF731FE046039
:100E5000A007BDE8F08746F48066E4E70028F8DAEA
:100E6000FFF726FE04606FF00040F2E7431A28BF48
:100E70009A427FF673AD104410F0030F11441EBF69
:100E800011F8013D521E00F8013D10F0030F7FF4F0
:100E9000F6AF103AC0F00A8010B531E91850103A98
:100EA00020E91850BFF4F9AFBDE81040530724BF44
:100EB00031E9081020E9081044BF51F8043D40F81A
:100EC000043D12F0030F08BF7047D20728BF31F866
:100ED000023D48BF11F8012C28BF20F8023D48BF51
:100EE00000F8012C7047000000487047086000209F
:100EF00010B500F085FC001D10BD00BFCD8A0000BC
:100F000030B5B0F10A024FEA900E71F100034EEADB
:100F1000817EB0EB0E0061EB91014FEA101E4EEAAC
:100F2000017E10EB0E0041EB11114FEA102E4EEA3C
:100F3000016E10EB0E0041EB11214FEA104E4EEA0C
:100F4000014E10EB0E0041EB1141401841F1000140
:100F50004FEAD00040EA41704FEAD10110EB800522
:100F60004FEA810444EA907444EB01046D1944EBA8
:100F70000404521BA3414FF0000348BF0A3200D5BE
:100F800030BD401C41F1000130BD70472DE9FF4FDD
:100F90000C461E464FF0FF378BB0D2E90001DDF85A
:100FA00060800A908A46C1F30A5505B93D46002182
:100FB00008464FF00000BAF1000F00F4400005DAD7
:100FC00000EB80004FF4400101EA50004FEA9059D5
:100FD000B9F1010F00DDB9460A9850EA4A000ED077
:100FE00044F61050A5F2FF3545432F14B8F1000F19
:100FF0001ED07542291E1EDDC9F100021CE0B8F1A9
:10100000010F4FF0000001D0302103E0F24305E072
:101010002154401CB042FBDB304600220021215409
:101020000B99C1F80880C1E900200FB0BDE8F08F2E
:10103000BD1B6D1CDEE74A4600DA694206A800F0D7
:1010400031FC06AB93E8070003AB83E8070050468A
:101050000A9900F0E3FC8DE80700A0F500501F3866
:1010600000900398002D0ADD42F21F014A46084411
:10107000002303A90390684600F04CFF09E0A0F5A7
:1010800000504A461F38002303A90390684600F029
:1010900056FF8DE807000004000C03D04FF0FF302E
:1010A000410800E01046B8F1000F03D00022009282
:1010B00015461EE0751E05D4FFF722FF303262553B
:1010C0006D1EF9D5B3460122084302D000227F1CD1
:1010D00004E02078302801D100227F1E002A0997E1
:1010E00084D01DE0112D07DAFFF70AFF3032625578
:1010F0006D1C50EA0102F5D1084302D00098C8B136
:101100000EE00021681E05E0235C625C63542254FB
:10111000401E491C8142F7DBAB46A81B401E0990CC
:10112000002004F80B000B98099AC0F80880C0E969
:10113000002B7AE711264FF0000857E72DE9F04F12
:1011400088460446D21D22F0070191B0D1E9000182
:10115000CDE90A0106F080FF02460B98C00F01D0CE
:101160002D2007E02068810701D52B2002E02021F7
:1011700001EAC000032A099001D0072A05DB0346D3
:101180004146204600F040FB0BE12078800601D567
:10119000E06900E00620B8F1650F814606D0B8F19D
:1011A000660F18D0B8F1670F70D131E00020B9F1A7
:1011B000110F009001DB112301E009F101030AAADC
:1011C00001A90CA8FFF7E2FEDDE90C70002609F189
:1011D0000105834647E001204B4600904FF0004751
:1011E0000AAA01A90CA8FFF7D1FEDDE90DB00C9900
:1011F0005D46002610B909F101000D18B9EB050094
:1012000003D4C0F1FF3609F10105A5EB09002BE07D
:10121000B9F1010F01DA4FF001090020B9F1110F06
:101220000090484601DD112300E003460AAA01A907
:101230000CA8FFF7ABFEDDE90C704D460026834697
:10124000207800070AD4AB4500DA5D4601A8012DDD
:1012500004DD411911F8011C302907D04F4502DA8D
:1012600017F1040F04DA012082460FE06D1EEEE74D
:10127000002F02DCED1B3E4403E0781CA84200DD99
:101280007D1CB81B00F1010A4FF0004720780007D1
:1012900003D4AA4501DB4FF0FF3A0021B7F1004F1C
:1012A0000DF143088DF8431024D002202B23002F8A
:1012B00001DA7F422D230A21021EA0F1010000DC89
:1012C0005FB197FBF1FC97FBF1F201FB1C7C174629
:1012D0000CF1300C08F801CDEEE7A8F10100037025
:1012E0002188090501D5452100E06521A0F101080B
:1012F00000F8011C09980FA9A1EB0807FF1D00B118
:101300000120411901EBEA70A1693844081A401E16
:10131000A0612078C00602D42046FFF73DF8099866
:1013200028B1D4E901219047206A401C206220782E
:10133000C00622D52046FFF72FF81EE0002E04DB62
:10134000B34502DD01A8805D00E03020D4E9012131
:101350009047206A401C2062761CAAF101005FEAD7
:10136000000A0AD100F04CFAC0680168405CD4E978
:1013700001219047206A401C2062281EA5F101052A
:10138000DCDC07E0D4E9012118F8010B9047206A62
:10139000401C2062381EA7F10107F3DC2046FFF74E
:1013A00011F8032011B041E62DE9F04F04460D4637
:1013B000D21D22F0070089B0D0E90097484639468F
:1013C00006F04AFE0246F80F01D02D2307E0206800
:1013D000810701D52B2302E0202101EAC0038DF80B
:1013E00020300BB1012000E00020032A824601D00A
:1013F000072A04DB2946204600F006FA3FE1207860
:10140000800601D40D2500E0E569C7F30A560D2DCD
:1014100049DA00214FEA175B08464FF00000002F21
:1014200000F4400007DA00EB80004FF4400100EBCD
:10143000D07001EA60008115012901DD4FF0FF3114
:1014400000224FEA850CBCF1180F06D31346ACF10D
:1014500018004FF08052C24003E04FF4801323FA8B
:101460000CF30CF10C0CBCF1200F04D3ACF1200CEC
:1014700009FA0CF001E007FA0CF000294FF00048DF
:1014800001DD18B90FE00ED140450CD319EB02096C
:101490005F4121B9404502D19F4329EA0209BBEBD4
:1014A000175F00D0761C2088000502D57B48784461
:1014B00002E07A487844193808AA302302F80A3042
:1014C000037C0AF10101002E0AF1020A53546A4614
:1014D00002DC4FF0300101E04FF031014FF0010824
:1014E0008DF8001002D0A6F2FF3603E059EA47015A
:1014F00000D06B4E002D02DC2178090704D54FF097
:1015000002082E218DF80110C44600210BE0C7F31C
:1015100003433F01C35C491C6D1E02F808300529D6
:1015200008F1010801DA002DF1DC00210CE000EBEC
:101530001973491C1B786D1E082902F808304FEA00
:10154000091908F1010801DA002DF0DC21688B0689
:1015500002D516E0A8F10108E04505DD02EB08031D
:1015600013F8013C302BF5D0B8F1000F09DD02EB88
:10157000080313F8013C2E2B03D1090701D4A8F16D
:101580000108002D05DD3E2102F808106D1E08F14E
:101590000108407C002E02F8080008F1010804DA76
:1015A0002D20764202F8080002E02B2002F8080005
:1015B0000A214FF47A70864208F101080BDB96FB92
:1015C000F0F3303302F8083096FBF0F308F101082D
:1015D00000FB136601E0642E0CDB642096FBF0F345
:1015E000303302F8083096FBF0F308F1010800FBF5
:1015F000136601E00A2E06DB96FBF1F0303002F8AC
:10160000080008F1010896FBF1F001FB1060303092
:1016100002F80800A16908F1010808EB050202EBD5
:101620000A00081AA0612078C00602D42046FEF7FE
:10163000B3FE216A08AE01EB0A00206204E0D4E99F
:10164000012116F8010B9047BAF1010AF7D2207870
:10165000C00602D52046FEF79FFE6E4609E016F84A
:10166000010B3E280FD0D4E901219047206A401C8D
:101670002062B8F10108F2D22046FEF7A3FE09B0BD
:101680000320BDE8F08F206A2844206203E0D4E9FB
:101690000121302090476D1EEBD3F8E79D880000B4
:1016A00002FCFFFF10B5436913B1AFF3008001E006
:1016B000FFF7D0FA012010BD128800F124018284C6
:1016C0000022C2840122EDE711684FF0FF32E9E702
:1016D0002DE9F05F824615468B4600270AF101048A
:1016E000B9460078302801D09DB113E014F8010B01
:1016F0000127782803D0582801D045B10AE00DB160
:10170000102D07D1002714F8010B102502E0082541
:1017100000E00A250026B0460EE005FB080005FBA8
:1017200006F101271FFA80F801EB1046B6F5803F5D
:1017300000D3B94614F8010B294600F0A5F800289B
:10174000EBDABBF1000F05D00FB1641E00E0544688
:10175000CBF80040B9F1000F06D0FFF7A9F902213C
:101760000160C81EBDE8F09F48EA0640FAE7007B2A
:1017700000F08000704770B516460C460546FFF72E
:10178000B7FB036893F80101012806D0FF2C0FD89E
:10179000185D68B101202C7070BDD3F80701324686
:1017A000214603F2071303442846BDE8704018475A
:1017B0004FF0FF3070BD7546FFF796FBAE46050053
:1017C0006946534620F00700854618B020B5FEF75D
:1017D00081FDBDE820404FF000064FF000074FF0BC
:1017E00000084FF0000B21F00701AC46ACE8C0093F
:1017F000ACE8C009ACE8C009ACE8C0098D46704748
:1018000000487047286000202DE9F0411F4604463B
:1018100003260168072A01F4006004DB08B116A55D
:1018200005E016A503E008B115A500E015A521F017
:1018300010002060A069C01EA0610FB1401EA06111
:101840002046FEF7A9FD4FB1D4E901213846904763
:10185000206A401C2062C01C206206E0206AFAE771
:10186000D4E9012115F8010B9047761EF8D22046E5
:10187000FEF7A8FDBDE8F0814E414E006E616E009E
:10188000494E4600696E66003A2800D2303820F092
:101890002002412A01D3A2F13700884201D34FF040
:1018A000FF3070472DE9F047814616468AB035482B
:1018B00078440DC88DE80D0032487844801C03AC94
:1018C0000DC884E80D0041F69B300844372190FB99
:1018D000F1F290FBF1F5A5F1800501FB12041B3C30
:1018E00002D56442012000E00020DFF898A0804685
:1018F0000027FA44AAF1BE0A0EE0E0070AD03246F9
:10190000684607EB470101230AEB810100F017FB52
:101910008DE8070064107F1C002CEED1194F7F4426
:10192000AE3F19E0E80715D007EB04100DF1180AD7
:1019300090E80E008AE80E00C068F04201D19819C4
:1019400008903246012306A903A800F0F8FA03AB79
:1019500083E807006D10641C002DE3D14FF00103F4
:1019600032466946B8F1000F03A802D000F0D2FA5F
:1019700001E000F0E4FAC9E90001C9F808200AB062
:10198000BDE8F0872C85000010B50446AFF3008059
:101990002046BDE81040FEF788BC00004FF0013C37
:1019A00050F8042B51F8043B9A4221D1A2EB0C03CE
:1019B000934313EACC1317D150F8042B51F8043B8E
:1019C0009A4215D1A2EB0C03934313EACC130BD12B
:1019D00050F8042B51F8043B9A4209D1A2EB0C03B6
:1019E000934313EACC13DBD04FF00000704700BFE5
:1019F000D01A01BAB1FA81F101F0180122FA01F00E
:101A0000CB40C1F12001DBB2C0B2C01A2CFA01F305
:101A1000D11A914311EAC311E6D170475FEA400C35
:101A200008BF91F0000F4FEA8C234FEAC12243EA2E
:101A300051514FEA1C5018BF00F5F0404FEA3000FA
:101A400018BF41F000415FEA6C5C00F02980BCF1F6
:101A5000FF3F08BF40F080407047130C06BF1204E0
:101A60004FF0100C4FF0000C130E04BF12020CF1DB
:101A7000080C130F04BF12010CF1040C930F04BFE8
:101A800092000CF1020CD30F04BF52000CF1010CB8
:101A900011464FF00002A0F11F00A0EB0C007047B0
:101AA00011F0004F08BF704731F000413FF4D5AF4F
:101AB0000B0C06BF09044FF0100C4FF0000C0B0E7E
:101AC00004BF09020CF1080C0B0F04BF09010CF153
:101AD000040C8B0F04BF89000CF1020CCB0F04BF68
:101AE00049000CF1010CCCF12003A0EB0C0022FA10
:101AF00003F302FA0CF241EA030100F1010070471E
:101B000020F07F4C80EA030023F07F47ACEB070313
:101B100003F57C5300F0004003F1FF032DE98049F9
:101B20004FEA154B09B44FEA144325EA0B4E24EA59
:101B300003480FF2042606EB132749083E785FEAB4
:101B4000320203FB0667C7F5000707FB06F64FEAFC
:101B500054374FEAD64606F1020607FB066CCCF175
:101B6000005C4FEA1C472CEA074C07FB06F40CFB11
:101B700006F504EB15464FEA961634BF00204FF0E9
:101B800000404FEAD13706FB07FC4FEA1C4C0CFB28
:101B90000BF7D21B03FB0CF761EB07010CFB0EF7F5
:101BA000B0EB074072EB17420CFB08F734BFA2EB17
:101BB0000742B2EB074261EB17414FEA0C444FEA90
:101BC000910706FB07FC4FEA1C4C0CFB0BF7B0EB34
:101BD000C74072EB573203FB0CF734BFA2EBC7428E
:101BE000B2EBC74261EB57310CFB0EF7B0EBC7000D
:101BF00072EB57720CFB08F734BFA2EBC702B2EBD3
:101C0000C70261EB5771039F4FEA816141EA92116C
:101C100004EBCC044FEAD1374FEA826206FB07FCA3
:101C200042EA90124FEA80604FEA1C4C0CFB0BF723
:101C3000D21B03FB0CF761EB07010CFB0EF7B0EBBB
:101C4000074072EB17420CFB08F734BFA2EB0742C8
:101C5000B2EB074261EB17414FEA8C554FEA91070F
:101C600004EB9C2406FB07FC4FEA1C4C0CFB0BF717
:101C7000B0EBC74072EB573203FB0CF734BFA2EB5B
:101C8000C742B2EBC74261EB57310CFB0EF7B0EB2A
:101C9000C70072EB57720CFB08F734BFA2EBC70208
:101CA000B2EBC70261EB577115EB4C254FEA81612E
:101CB00041EA92114FEA82624FEAD13742EA90122A
:101CC00006FB07FC44F100044FEA80604FEA1C4C1D
:101CD0000CFB0BF7D21B03FB0CF761EB07010CFBB2
:101CE0000EF7B0EB074072EB17420CFB08F734BF5E
:101CF000A2EB0742B2EB074261EB174115EB1C1553
:101D00004FEA813141EA92414FEA823242EA9042FF
:101D10004FEA80304FEA0C7644F1000448EA03436E
:101D20004EEA0B484FF0000EB2EB080C71EB0307C4
:101D300024BF624639464EEB0E0E4FF0000B0018E2
:101D4000524149414BEB0B0BB2EB080C71EB030713
:101D50007BF1000B24BF624639464EEB0E0E4FF06E
:101D6000000B0018524149414BEB0B0BB2EB080C36
:101D700071EB03077BF1000B24BF624639464EEB43
:101D80000E0E51EA020718BF46F0010616EB0E765A
:101D900055F1000254F1000103D5BDE88901BDE809
:101DA0000088BDE88901BDE80048B619524141EB01
:101DB0000101A3F10103704780807F7E7D7C7B7AE7
:101DC0007978777676757473727171706F6E6E6DE7
:101DD0006C6C6B6A6A69686867666665646463638D
:101DE00062616160605F5F5E5E5D5D5C5C5B5B5A13
:101DF0005A59595858575756565555555454535380
:101E000052525251515050504F4F4F4E4E4D4D4DDA
:101E10004C4C4C4B4B4B4A4A4A4949494848484725
:101E20004747474646464545454444444443434363
:101E30004342424242414141002B9C4630D477000C
:101E40002BD01CB54FEA370703B44FF010004FF00A
:101E50001001BAF1000F06D0BCF1000FDCBF40F05A
:101E6000080040F008014FF000000FBCBDE8104032
:101E70000BF1010BBBF1010F08BF5FEA170722BF8F
:101E800012F1010211F101014FF0004143F1000391
:101E900000F0004043EA00007047F9D35708D0E74C
:101EA00046EA064613F1400F4FEA16461FDD13F1CE
:101EB000200FDFBF16430A46002120335B42BED00D
:101EC000C3F1200746EA064602FA07F74FEA16462C
:101ED00046EA0706C3F1200722FA03F201FA07F7E0
:101EE00021FA03F14FF0000342EA0702A7E746EAAE
:101EF000020646EA06464FEA164646EA0106BCBF17
:101F000046EA0646360C4FF000034FF000024FF051
:101F1000000194E72DE9804C9A46934670B491E80D
:101F2000380007C831EA400C48BF34EA430C03D5F7
:101F3000FFF7E6FDFFF780FFF0BCBDE8008C2DE960
:101F4000804C9A46934670B491E8380007C810F068
:101F5000804F08BF13F0804F03D100F005F8FFF762
:101F60006BFFF0BCBDE8008C20F07F4780EA0300E7
:101F700023F07F4C07EB0C03A3F57C5300F00040EB
:101F8000A3F1FE0392F0000F00F0B38095F0000F74
:101F900000F077802DE901494FEA11404FEA1446DD
:101FA00021EA004800FB06FC24EA064708FB06F687
:101FB00007FB08F800FB07F718EB06484CEB164C3C
:101FC0004FEA124B18EB07484FEA15464CEB174007
:101FD00022EA0B4E0BFB06FC25EA06470EFB06F633
:101FE00007FB0EFE0BFB07F71EEB064E4CEB164CE9
:101FF0004FF000061EEB074E4CEB174B18EB0B088F
:1020000040F1000018EB0E0B58EB000840F1000007
:102010008F1A4FF000013CBFC943661B14BFB5EBDC
:10202000040C00213CBFC943F61B4FEA17444EEA9B
:102030008E0E27EA04454FEA1C4704FB07622CEA90
:10204000074C05FB07F70CFB05F604FB0CFC16EB35
:10205000074642EB174216EB0C4642EB1C421BEBC9
:10206000060658EB0202414146EA9E0601D5BDE84C
:102070000189B619524141EB0101A3F10103BDE809
:1020800001894FEA14454FEA114724EA054621EA3F
:10209000074C05FB07F406FB07F70CFB06F105FBF5
:1020A0000CFC11EB074144EB17444FEA124711EBCC
:1020B0000C4144EB1C4422EA074C05FB07F206FBEB
:1020C00007F70CFB06F605FB0CFC16EB074642EB8C
:1020D000174216EB0C4642EB1C456A1854F10001FE
:1020E00048BF7047B619524141EB0101A3F101030A
:1020F000704795F0000F37D04FEA11424FEA14476E
:1021000021EA024624EA074C02FB07F106FB07F727
:102110000CFB06F402FB0CFC14EB074441EB1741EB
:102120004FEA154714EB0C4441EB1C4125EA074CE0
:1021300002FB07F506FB07F70CFB06F602FB0CFC9F
:1021400016EB074645EB174516EB0C4645EB1C42D4
:10215000121951F1000148BF7047B619524141EBC5
:102160000101A3F1010370474FEA14454FEA1147FB
:1021700024EA054621EA074C05FB07F106FB07F7B1
:102180000CFB06F24FF0000605FB0CFC12EB0742BD
:1021900041EB174112EB0C4251EB1C4148BF704719
:1021A000921841EB0101A3F10103704770B5044699
:1021B00000252068806800F00100F0B12068806888
:1021C00020F001002168886002F012F805460EE058
:1021D00002F00EF8401B022809D9A06A40F0100056
:1021E000A062E06A40F00100E062012070BD20685A
:1021F000806800F001000028EAD10020F6E7000026
:1022000038B504460025002000902068806800F062
:10221000010080BB2068806840F001002168886070
:10222000164800681649B0FBF1F0009002E00098F3
:10223000401E009000980028F9D101F0D9FF054612
:1022400013E001F0D5FF401B02280ED9A06A40F030
:102250001000A062E06A40F00100E06200BF0020D0
:1022600084F8240000BF012038BD2068806800F099
:1022700001000028E5D00020F6E70000080000205B
:1022800040420F0000BFFEE7704710B5012001F08B
:10229000EBFD10BD0021074AD1610749096941F0F2
:1022A0000401054A11611146096941F040011161BB
:1022B00070470000804A0020002002400021074AA9
:1022C000D1610749096941F00201054A11611146CE
:1022D0004861096941F0400111617047804A00205E
:1022E000002002400022054BDA61054A126942F0E3
:1022F0000102034B1A61018070470000804A0020F0
:102300000020024000201E49C96801F0100139B1C7
:102310001C49C96941F002011A4AD16140F010001C
:102320001749C96801F0040139B11649C96941F07A
:102330000101144AD16140F004001149C96901F05A
:10234000010169B10F49C96941F004010D4AD16128
:1023500000BF0B49C96921F00101094AD16100BFE1
:1023600000BF40F20111884206D10549C96921F038
:102370000101034AD16101E00149C86000BF704713
:1023800000200240804A002070B5044601F030FF72
:10239000054609E0601C38B124B101F029FF401B5B
:1023A000A04201D9032070BD1248C06800F00100AE
:1023B0000028EFD10F48C06800F0200020B100BF16
:1023C00020200C49C86000BF0A48C06800F0100017
:1023D00048B90848C06900F0010020B90548C06844
:1023E00000F0040018B1FFF78DFF0120DBE70020AB
:1023F000D9E70000002002402DE9F04105460F46D4
:102400001A4807601A480068A8422CD00026002409
:102410001748056017A1284605F021FB044608E08F
:1024200020785C2802D020782F2801D1641C02E09B
:10243000641EAC42F4D100BF0DE0202E06DA14F881
:10244000012B3046761C0C490A5404E000200A494E
:102450000870002602E020780028EED100BF00209E
:102460000549885500BF0120BDE8F08140260020C5
:102470003C2600202E6300003053002077B585B045
:1024800004460D4600200290039004904FF4C06172
:102490002448FEF795FA022C14D0032C0DD0042CFE
:1024A00006D0052C13D120A102A805F0CBFA13E029
:1024B0001EA102A805F0C6FA0EE01DA102A805F0B3
:1024C000C1FA09E01BA102A805F0BCFA04E01AA1B8
:1024D00002A805F0B7FA00BF00BF18480068184B03
:1024E00002AA18A100900F4803F022F90D48FEF748
:1024F00038F90C4946182A464FF4C0713046079BFC
:1025000003F01EFD12A10748FEF795F90548FEF7F6
:1025100028F9C6B2314603480E4A1268904708B0FF
:1025200070BD0000304D0020440000004900000054
:102530005700000045000000460000004026002033
:10254000305300205B25735D5B25733A25645D0085
:102550000D0A0000442600203EB5044600940120E8
:102560000190072002906946074800F091F806485C
:1025700000F0D8FA0A21044800F01CFA024800F0E2
:1025800037F980B23EBD00009C4C0020F8B50446EF
:1025900000260020009000BF94F82400012801D1FB
:1025A0000220F8BD012084F8240000BF2046FFF778
:1025B000FDFD0646002E62D1A06A20F4885040F04E
:1025C0000200A062022001F053FF30490968B1FB0C
:1025D000F0F04000009002E00098401E009000984B
:1025E0000028F9D12046FFF70BFE2068806840F0F4
:1025F00008002168886001F0FBFD054611E001F04C
:10260000F7FD401B0A280CD9A06A20F0020040F018
:102610001000A06200BF002084F8240000BF012049
:10262000BFE72068806800F008000028E7D1206834
:10263000806840F004002168886001F0D9FD0546FB
:1026400011E001F0D5FD401B0A280CD9A06A20F04A
:10265000020040F01000A06200BF002084F82400B7
:1026600000BF01209DE72068806800F0040000287A
:10267000E7D1A06A20F0020040F00100A06200BF94
:10268000002084F8240000BF30468AE708000020BC
:1026900038B5024600230020009000BF92F82400C5
:1026A000012801D1022038BD012082F8240000BF9A
:1026B0004868072812D21068406B0C79641E04EB3E
:1026C00084051F24AC40A0430D796D1E05EB8505E4
:1026D0000C68AC4020431468606327E048680D280C
:1026E00012D21068006B0C79E41F04EB84051F24E0
:1026F000AC40A0430D79ED1F05EB85050C68AC409F
:1027000020431468206311E01068C06A0C790D3C06
:1027100004EB84051F24AC40A0430D790D3D05EB6F
:1027200085050C68AC4020431468E06208680A28FC
:1027300012D31068C0680C780A3C04EB44050724E7
:10274000AC40A0430D780A3D05EB45058C68AC40D4
:1027500020431468E0600FE0106800690C7804EB17
:1027600044050724AC40A0430D7805EB45058C6873
:10277000AC402043146820610868102802D0086823
:10278000112827D1174C1068A0421ED1106880680C
:1027900000F40000F0B91068806840F4000014688C
:1027A000A0600868102815D10F4800680F4CB0FBD6
:1027B000F4F000EB80004000009002E00098401E22
:1027C000009000980028F9D104E0906A40F02000C1
:1027D0009062012300BF002082F8240000BF184649
:1027E00061E70000002401400800002040420F0083
:1027F00001460868C06C70472DE9F0410446002787
:1028000000250026A84614B90120BDE8F081A06883
:1028100010B1207D00B100BFA06A30B90020E06295
:1028200084F82400204600F097F82046FFF7BEFC0D
:102830000746A06A00F01000002873D1002F7ED157
:10284000A06A20F4885040F00200A0623F4AD4E918
:102850000001904208D1E069B0F5402F02D14FF459
:10286000002002E0E06900E0E0690143207B41EAEA
:1028700040000643A068B0F5807F02D0A068012820
:1028800002D14FF4807000E000200543207D012834
:1028900011D1207B38B9A069401E4FF4006141EA94
:1028A0004030054307E0A06A40F02000A062E06AE3
:1028B00040F00100E0622068406820F4694028434D
:1028C00021684860206880682149084030432168B9
:1028D0008860A068B0F5807F02D0A068012802D18E
:1028E0004FF4807000E00020B0F5807F03D1208A93
:1028F000401E4FEA00582068C06A20F4700040EA89
:1029000008002168C8622068806812490840B04207
:1029100009D10020E062A06A20F0020040F001002E
:10292000A06211E00BE0A06A20F0020040F010006D
:10293000A062E06A40F00100E062012704E0A06AC2
:1029400040F01000A062012738465EE7003C0140DD
:10295000FDF7E1FFFE0E1FFF10B586B0044600BF75
:102960001248806940F40070104988610846806907
:1029700000F40070019000BF00BF00BF08468069EE
:1029800040F0040088610846806900F0040001906E
:1029900000BF00BF0220029003200390002004909B
:1029A00002A9034801F06EFA06B010BD0010024003
:1029B00000080140F8B504460D46002600200090AE
:1029C000002701F015FC06462068806800F480703E
:1029D00050B1A06A40F02000A06200BF002084F83F
:1029E000240000BF0120F8BD2068406800F480701A
:1029F000F8B92068C06A00F47000D0B912E0681C11
:102A000080B125B101F0F4FB801BA8420AD9A06A6D
:102A100040F00400A06200BF002084F8240000BF42
:102A20000320E0E72068006800F002000028E6D0FC
:102A300050E0022001F01CFD36490968B1FBF0F0BE
:102A400021680969344A114091B92168C968921115
:102A5000114069B921680969304A114031B92168CA
:102A6000C9689211114009B9142117E0292115E014
:102A700021680969294A114021B92168C968921160
:102A8000114041B121680969254A114029B92168DD
:102A9000C968114009B9542100E0FC2100FB01F78D
:102AA00015E0681C80B125B101F0A2FB801BA84293
:102AB0000AD9A06A40F00400A06200BF002084F898
:102AC000240000BF03208EE70098401C009000986F
:102AD000B842E6D36FF0120021680860A06A40F4A3
:102AE0000070A0622068806800F46020B0F5602F5C
:102AF0000DD1207B58B9A06A20F48070A062A06A32
:102B000000F4805018B9A06A40F00100A0620020D3
:102B100069E7000008000020244992249224491209
:102B20004992240070B50446002500BF94F82400A3
:102B3000012801D1022070BD012084F8240000BFCB
:102B40002046FFF75DFB0546002D77D1A06A40F2D5
:102B50000121884340F48070A0623C49206888428B
:102B600008D13B48006800F4702008B9012002E059
:102B7000002000E0012078B1A06A20F48010A0625B
:102B80002068406800F4806000B3A06A20F4005020
:102B900040F48050A06219E0A06A40F48010A06266
:102BA0002B49091F2068884203D0284920688842A1
:102BB00004D12748006800F4806000E0002028B1BC
:102BC000A06A20F4005040F48050A062A06A00F493
:102BD000805020B1E06A20F00600E06201E00020B1
:102BE000E06200BF002084F8240000BFC01E2168FE
:102BF00008602068806800F46020B0F5602F16D16E
:102C000012492068884208D11148006800F47020F9
:102C100008B9012002E0002000E0012038B120685E
:102C2000806840F4A000216888600CE006E020681D
:102C3000806840F480102168886004E000BF0020B4
:102C400084F8240000BF284675E7000000280140F2
:102C50000424014070B50024002508E00120FFF79E
:102C60007BFC0444032005F0E5FA681CC5B2032D83
:102C7000F4DB0320B4FBF0F080B270BD00B587B088
:102C8000022001908003039001A801F08BFC0C4806
:102C90000C4908600020486000210A4881600173E7
:102CA000012101610021017581614FF46021C16141
:102CB000FFF7A2FD0348FFF769FC07B000BD000065
:102CC000002401409C4C002000B585B000BF0F4897
:102CD000806940F004000D4988610846806900F071
:102CE0000400009000BF00BF01200290022003906A
:102CF00004900820019001A9054801F0C3F80022C2
:102D00000821034801F06DFA05B000BD0010024033
:102D10000008014010B504462CB1012208210548E5
:102D200001F05FFA04E000220821024801F059FA9C
:102D300010BD00000008014010B50020FFF7EAFFB9
:102D400002F0EEFC002002F0C7FC02F07BFCC82081
:102D500005F070FA0120FFF7DDFF02F095FC01207D
:102D600002F0BAFC10BD10B5024692F82030012BDB
:102D700001D0022B06D110684069084314686061D5
:102D8000002010BD506A40F4802050620120F8E716
:102D9000F0B504460D461E4694F8207020688368FE
:102DA000A86800B900E000BF012F01D0022F7CD13C
:102DB00003F0806030B903F0006018B903F0805070
:102DC000002873D0C3F30161022905D9606A40F479
:102DD000000060620120F0BD012088403060A868DA
:102DE00060B9B5F800C0E86840EA4C5C206800F5BE
:102DF000C07000EB0110C0F800C00FE0D5E901C0C1
:102E000040EACC00D5F80CC040EA0C00D4F800C071
:102E10000CF5C07C0CEB011CCCF80000D5F810C000
:102E2000206800F5C07000EB0110C0F804C0287DD8
:102E300001280ED1206800F5C07000EB0110406839
:102E400040F4807C206800F5C07000EB0110C0F8F1
:102E500004C0D079000692F806C040EA0C4092F80F
:102E600005C040EA0C2C10794CEA000C206800F5F3
:102E7000C07000EB0110C0F80CC0D078000692F8CA
:102E800002C040EA0C4092F801C040EA0C2092F8DF
:102E900000C040EA0C00D4F800C00CF5C07C0CEB7C
:102EA000011CCCF80800206801E016E00FE000F5F6
:102EB000C07000EB0110006840F0010C206800F5C4
:102EC000C07000EB0110C0F800C0002083E7606A0A
:102ED00040F40010606201207DE7606A40F48020C9
:102EE0006062012077E7F0B504460A46216894F84D
:102EF0002050012D01D0022D74D1D1F8000240F0F4
:102F00000100C1F80002107D00F01F06012000FA48
:102F100006F3D1F81C029843C1F81C02D069C8B965
:102F2000D1F80C029843C1F80C02908880B29689BF
:102F300040EA064601F51070576940F8376010887E
:102F400080B2168940EA064601F51070576900EB19
:102F5000C7004660D069012819D1D1F80C02184386
:102F6000C1F80C02908880B2168840EA064601F546
:102F70001070576940F83760908980B2168940EA2E
:102F8000064601F51070576900EBC700466090696E
:102F900028B9D1F804029843C1F8040204E0D1F83A
:102FA00004021843C1F80402106928B9D1F81402C8
:102FB0009843C1F8140204E0D1F814021843C1F890
:102FC0001402106A012804D1D1F81C021843C1F878
:102FD0001C02D1F8000220F00100C1F8000200201C
:102FE000F0BDFFE7606A40F4802060620120F7E7EF
:102FF0002DE9FF47044620688069050E2068806936
:10300000C0F3074620688069C0F302172068806912
:1030100000F0010820688069C0F3400920688069D9
:10302000C0F3800A40F2191110A0FFF7E5F938B19A
:103030008DE88007616A33462A46134804F0D8FFBA
:1030400012480078401C1149087008460078022890
:1030500003DA0F490F4800F059FC0F48006818B117
:10306000606A0D4909688847BDE8FF872E2E5C48D5
:10307000415244574152455C43414E5C68616C5F2C
:1030800063616E2E63000000F89D00084000002080
:1030900038000020D04B00203000002070B50446DE
:1030A00094F82050012D01D0022D7DD151B9206816
:1030B000C06800F0030080B9606A40F400106062EC
:1030C000012070BD2068006900F0030028B9606A23
:1030D00040F4001060620120F3E7206800F5D8702A
:1030E00000EB0110006800F004009060906840B9A7
:1030F000206800F5D87000EB01100068400D1060EA
:1031000007E0206800F5D87000EB01100068C008E7
:103110005060206800F5D87000EB0110006800F0E6
:103120000200D060206800F5D87000EB0110406804
:1031300000F00F001061206800F5D87000EB01105E
:10314000406800F47F40000A9061206800F5D87064
:1031500000EB01104068000C5061206800F5D87049
:1031600000EB011080681870206800F5D87000EB43
:103170000110806800F47F40000A5870206800F554
:10318000D87000EB0110806800F47F00000C98708C
:10319000206800F5D87000EB01108068000ED87030
:1031A000206800F5D87000E02FE000EB0110C06847
:1031B0001871206800F5D87000EB0110C06800F4A9
:1031C0007F40000A5871206800F5D87000EB0110AC
:1031D000C06800F47F00000C9871206800F5D8707A
:1031E00000EB0110C068000ED87131B92068C068CA
:1031F00040F020002668F06005E02068006940F09B
:1032000020002668306100205BE7606A40F480207F
:103210006062012055E72DE9F05F04460025206833
:1032200046692068D0F80490206887682068D0F844
:103230000CA02068D0F810B02068D0F8188006F0F4
:103240000100002855D007F00100C0B1012021681D
:10325000886007F0020018B1204600F08FFA0EE0F7
:1032600007F0040010B145F4006508E007F008001D
:1032700010B145F4805502E0204600F07DFA07F4D5
:103280008070C8B14FF480702168886007F40070C6
:1032900018B1204600F080FA0EE007F4806010B10B
:1032A00045F4005508E007F4006010B145F480458E
:1032B00002E0204600F06EFA07F48030C8B14FF407
:1032C00080302168886007F4003018B1204600F093
:1032D00071FA0EE007F4802010B145F4004508E0D3
:1032E00007F4002010B145F4803502E0204600F0DC
:1032F0005FFA06F0080038B10AF0100020B145F47A
:10330000007510202168C86006F0040040B10AF082
:10331000080028B108202168C860204600F0A8F9FC
:1033200006F0020038B12068C06800F0030010B158
:10333000204600F09FF906F0400038B10BF0100075
:1033400020B145F4806510202168086106F0200056
:1033500040B10BF0080028B1082021680861204620
:1033600000F0D8F906F0100038B12068006900F0CC
:10337000030010B1204600F0CEF906F4003040B151
:1033800009F0100028B1102021684860204600F0A4
:10339000C3F906F4803040B109F0080028B10820D4
:1033A00021684860204600F011FA06F4004088B316
:1033B00009F0040078B306F4807020B108F0010031
:1033C00008B145F0010506F4007020B108F00200D4
:1033D00008B145F0020506F4806020B108F0040051
:1033E00008B145F0040506F40060A0B108F07000D3
:1033F00088B108F07000402817D006DC10280BD0E8
:1034000020280CD0302819D10CE0502810D060288A
:1034100014D110E01DE019E045F008050FE045F07B
:1034200010050CE045F0200509E045F0400506E0F8
:1034300045F0800503E045F4807500E000BF00BF63
:103440002068806920F0700021688861042021686C
:1034500048602DB1606A284360622046FFF7C8FDCE
:10346000BDE8F09F70B504460CB9012070BD94F81A
:10347000200010B9204600F0AFF82068006820F066
:1034800002002168086000F0B3FE05460DE000F080
:10349000AFFE401B0A2808D9606A40F40030606221
:1034A000052084F820000120E0E72068406800F053
:1034B00002000028EBD12068006840F0010021687C
:1034C000086000F095FE05460DE000F091FE401BFF
:1034D0000A2808D9606A40F400306062052084F848
:1034E00020000120C2E72068406800F001000028A9
:1034F000EBD0207E012806D12068006840F08000D3
:103500002168086005E02068006820F080002168DC
:103510000860607E012806D12068006840F0400005
:103520002168086005E02068006820F040002168FC
:103530000860A07E012806D12068006840F02000C5
:103540002168086005E02068006820F020002168FC
:103550000860E07E012806D12068006820F0100095
:103560002168086005E02068006840F010002168CC
:103570000860207F012806D12068006840F008001C
:103580002168086005E02068006820F008002168D4
:103590000860607F012806D12068006840F00400C0
:1035A0002168086005E02068006820F004002168B8
:1035B0000860D4E9020108432169084361690843AE
:1035C0006168491E08432168C861002060620120CB
:1035D00084F82000002049E710B586B0044600BFFB
:1035E0002148C06940F000701F49C8610846C069A1
:1035F00000F00070019000BF00BF00BF0846806966
:1036000040F0040088610846806900F004000190E1
:1036100000BF00BF88140290022003900120049094
:103620000320059002A9114800F02CFC4FF4006023
:103630000290002003900320059002A90B4800F09F
:1036400021FC00220821142000F0BFFE142000F00D
:10365000ACFE00220821132000F0B7FE132000F07A
:10366000A4FE06B010BD000000100240000801409A
:103670007047000030B589B004461C2102A8FDF750
:10368000C1F90020009001906B4602AA002120465B
:10369000FFF704FDE0B913480068002820D0049823
:1036A00048B9069AD3B2049AD0B26A460D4D02992F
:1036B0002D68A84714E00498042811D1069AD3B2C3
:1036C000DDE90312D0B26A46064D2D68A84707E02F
:1036D000F52105A0FEF790FE10B10AA004F088FCC9
:1036E00009B030BD280000202E2E5C4841524457BE
:1036F0004152455C43414E5C68616C5F63616E2E74
:1037000063000000476574205278204D73672045A0
:103710005252000070477047704770B5044694F8E5
:103720002000012822D1022084F8200020680068AF
:1037300020F001002168086000F05AFD05460DE008
:1037400000F056FD401B0A2808D9606A40F400309A
:103750006062052084F82000012070BD2068406868
:1037600000F001000028EBD16062F6E7606A40F4E7
:10377000002060620120F0E77047000010B50446A9
:103780000348006810B102480068804710BD00007F
:103790002C0000207047000010B504460348006864
:1037A00010B102480068804710BD00002C000020C6
:1037B0007047000010B504460348006810B1024885
:1037C0000068804710BD00002C00002070470000FA
:1037D00008B101B102B97047034B1860034B19607F
:1037E000034B1A6000BFF6E7280000202C000020E1
:1037F0003000002010B58AB000200590069001200E
:103800000790002000900190029003900490012006
:1038100008900E20099069460548FFF764FB0446AE
:103820001CB14FF0FF300AB010BD0020FBE70000D4
:10383000A84B002010B52D482D49086000212C48C8
:10384000017641768176C176017741778160C160EA
:103850000420274948604104254801614FF4E001F4
:103860004161FFF7FFFD044614B14FF0FF3010BD7A
:10387000FFF7C0FF044614B16FF00100F7E7022123
:103880001B48FFF770FA10B16FF00200EFE701215B
:103890001748FFF768FA10B16FF00200E7E74FF43E
:1038A00080611348FFF75FFA10B16FF00200DEE7A6
:1038B0004FF480710E48FFF756FA10B16FF0020016
:1038C000D5E74FF400710A48FFF74DFA10B16FF0D9
:1038D0000200CCE74FF400410548FFF744FA10B16D
:1038E0006FF00200C3E70020C1E700000064004061
:1038F000A84B002010B50448FFF70FFF10B14FF0A0
:10390000FF3010BD0020FCE7A84B002070B5044636
:103910000D46064B2A4621460548FFF739FA10B1F5
:103920004FF0FF3070BD0020FCE7000034000020A5
:10393000A84B00202DE9F84304460D4616461F46C5
:103940001EB94FF0FF30BDE8F88300202849087009
:10395000A52128A0FEF750FD58B13946304603F0A6
:1039600073FF81463B462A462146009028A004F07A
:1039700059FB3CB9002034498860084605600020A6
:1039800048600CE0042C07D104202F4988600020F7
:1039900008600846456002E06FF00100D3E7082F99
:1039A00001DD082000E03846804600202649C86036
:1039B0000846C0F8108000200875244800210160E6
:1039C000416042463146FCF742FF20491E48FFF75E
:1039D0009DFF50B1C22107A0FEF70EFD10B11CA043
:1039E00004F006FB6FF00200ADE70020ABE700003B
:1039F000400000202E2E5C48415244574152455C05
:103A000043414E5C68616C5F63616E2E6300000031
:103A100074782063616E5F69645F747970653A25BC
:103A2000642C63616E5F69642C307825782C70613A
:103A3000796C6F61645F6C656E3A25642C70617996
:103A40006C6F61643A257300D04B00203800002071
:103A500048414C5F43616E5478206572726F72000A
:103A600070B50446002594F82100022803D00420F4
:103A7000A0630125C1E02068006820F00E002168E5
:103A800008602068006820F00100216808605C4937
:103A90002068884252D95A4978392068884201D131
:103AA000012047E0564964392068884201D110203E
:103AB00040E0534950392068884201D1801539E0EF
:103AC0004F493C392068884201D1801432E04C498A
:103AD00028392068884202D14FF480302AE04849D2
:103AE00014392068884202D14FF4801022E0444902
:103AF0002068884201D140041CE042492068884285
:103B000001D1012016E03F4914312068884201D1DB
:103B100010200FE03B4928312068884201D18015F0
:103B200008E038493C312068884201D1801401E026
:103B30004FF480303349091F086051E0304978392B
:103B40002068884201D1012047E02D49643920686E
:103B5000884201D1102040E029495039206888422C
:103B600001D1801539E026493C392068884201D1CD
:103B7000801432E0224928392068884202D14FF46B
:103B800080302AE01E4914392068884202D14FF45F
:103B9000801022E01A492068884201D140041CE0CC
:103BA00018492068884201D1012016E015491431D6
:103BB0002068884201D110200FE012492831206886
:103BC000884201D1801508E00E493C3120688842C6
:103BD00001D1801401E04FF48030094980394860F8
:103BE000012084F8210000BF002084F8200000BFDD
:103BF000606B10B12046616B8847284670BD00009D
:103C000080000240080402402DE9F04104460E46BF
:103C10000127002500BF2648007E012802D102208E
:103C2000BDE8F08101202249087600BF2068022803
:103C300013D14CF25030FEF7A7FB90BB0120FEF7EA
:103C400029FB4CF25030FEF79FFB074619480069EC
:103C500020F004001749086123E04CF25030FEF7D1
:103C600093FBF0B94FF0FF303060A56812E02846B2
:103C7000FEF724FB4CF25030FEF786FB07460D485A
:103C8000006920F002000B4908610FB1356007E0C0
:103C900005F50065D4E9021001EBC020A842E6D882
:103CA00000BF00BF00200249087600BF3846B7E7D2
:103CB000804A0020002002400348006940F0800054
:103CC0000149086100207047002002402DE9FE4FA5
:103CD00005468B4617469846012600240020029090
:103CE00000BF2448007E012802D10220BDE8FE8FDB
:103CF00001202049087600BF4CF25030FEF744FB0B
:103D0000064686BB012D02D10120029006E0022D5D
:103D100002D10220029001E00420029000241EE063
:103D20002201B946C24648465146FCF7E6FA80B23F
:103D30000190022000FB04B000900199FEF7D2FA36
:103D40004CF25030FEF720FB06460B48006920F08D
:103D500001000949086106B104E0601CC4B2029880
:103D60008442DDDB00BF00BF00200249087600BFAF
:103D70003046BBE7804A002000200240002008496E
:103D8000096901F0800151B10649054A51600649AF
:103D900051601146096901F0800101B101207047AD
:103DA0000020024023016745AB89EFCD014600208A
:103DB000704770B504460D461646324621462846E1
:103DC000FCF745FD002070BD10B50446204604F008
:103DD00073F910BD2DE9F84F06460F4690464FEA9D
:103DE000A80BA8EB8B000090002400250BE057F8EF
:103DF00005A07019514604F081F910B10120BDE809
:103E0000F88F2D1D641C5C45F1DB0098B8B14FF0B4
:103E1000000AD146002408E07819005D00FA09F094
:103E200040EA0A0A09F10809641C00988442F3DB9D
:103E30007019514604F062F908B10120DFE7002053
:103E4000DDE7000010B50446012C07D105480068E5
:103E500018B1002003490968884700E000BF00BF8F
:103E600010BD00004400002010B50446044800685E
:103E7000204020B1024804602046FFF7E3FF10BD58
:103E8000140401402DE9F847024600239C467BE1DB
:103E90004FF0010808FA03F4D1F8008008EA0400A2
:103EA000A0427DD1DFF8F4A2D1F80480A8EB0A0982
:103EB000D0453AD014DCB8F1030F50D009DCB8F18A
:103EC000000F31D0B8F1010F1CD0B8F1020F49D169
:103ED00020E0B8F1110F18D0B8F1120F42D11EE056
:103EE000B9F5881F25D006DCB9F5803F20D0B9F59B
:103EF000801F37D11AE0B9F5001F18D0B9F5041F9B
:103F000030D117E0D1F80CC02DE0D1F80C8008F1C9
:103F1000040C28E0D1F80C8008F1080C23E0D1F85B
:103F20000C8008F10C0C1EE000BF00BF00BF00BFFA
:103F300000BF00BFD1F80880B8F1000F02D14FF0E8
:103F4000040C0BE0D1F80880B8F1010F03D14FF059
:103F5000080C146102E04FF0080C546103E04FF0CC
:103F6000000C00E000BF00BFFF2801D8904601E030
:103F700002F104084646FF2802D84FEA830803E00E
:103F8000A3F108084FEA88084746D6F800804FF0AA
:103F90000F0909FA07F928EA09080CFA07F900E0FD
:103FA0007AE048EA0908C6F80080D1F8048008F0F1
:103FB0008058B8F1805F6FD100BFDFF8E481D8F896
:103FC000188048F00108DFF8D891C9F81880C84671
:103FD000D8F8188008F00108CDF8008000BF00BFB5
:103FE0004FEAB9384FEA930958F829504FEA8378D5
:103FF0004FEA18794FF00F0808FA09F825EA080582
:10400000DFF8A081424502D14FF0000824E0DFF83C
:104010009881424502D14FF001081DE0DFF88C8104
:10402000424502D14FF0020816E0DFF88481424594
:1040300002D14FF003080FE0DFF87881424502D14A
:104040004FF0040808E0DFF87081424502D14FF0DC
:10405000050801E04FF006084FEA83794FEA197925
:1040600008FA09F848EA0505DFF850814FEA930994
:1040700048F82950D1F8048008F48038B8F5803F1A
:104080000BD1DFF83C81D8F8008048EA0008DFF85F
:104090003091C9F800800AE075E0DFF82481D8F893
:1040A000008028EA0008DFF81891C9F80080D1F8EC
:1040B000048008F40038B8F5003F0ED1DFF8008125
:1040C00008F10408D8F8008048EA0008DFF8F0900A
:1040D00009F10409C9F800800DE0DFF8E48008F177
:1040E0000408D8F8008028EA0008DFF8D49009F125
:1040F0000409C9F80080D1F8048008F48018B8F5E4
:10410000801F0ED1DFF8B88008F10808D8F80080C9
:1041100048EA0008DFF8A89009F10809C9F800800A
:104120000DE0DFF89C8008F10808D8F8008028EA44
:104130000008DFF88C9009F10809C9F80080D1F86F
:10414000048008F40018B8F5001F0ED1DFF8708065
:1041500008F10C08D8F8008048EA0008DFF8609001
:1041600009F10C09C9F800800DE0DFF8548008F16E
:104170000C08D8F8008028EA0008DFF8449009F11C
:104180000C09C9F800805B1CD1F8008028FA03F8FC
:10419000B8F1000F7FF47CAEBDE8F8870000111085
:1041A0000010024000080140000C014000100140D6
:1041B0000014014000180140001C014008000140AB
:1041C00000040140024693680B400BB1012000E05F
:1041D00000207047C2680A400AB1416100E00161F5
:1041E00070470AB1016101E00B04036170470000F0
:1041F00001480068704700000C00002070B50446BC
:104200000CB9012070BD4CF6CC402168086045F225
:10421000555021680860D4E9001048602168A06802
:104220008860FFF7E5FF054606E0FFF7E1FF401B6A
:10423000302801D90320E5E72068C0680028F4D1C0
:104240004AF6AA20216808600020DBE701464AF60A
:10425000AA200A6810600020704700000348006828
:104260000349097808440149086070470C000020A0
:104270001400002010B50848006840F010000649FE
:104280000860052000F0E0F80F2000F007F800F0CB
:104290008BF8002010BD00000020024070B50446DD
:1042A0000E4800784FF47A71B1FBF0F00C490968C0
:1042B000B1FBF0F5284601F0AAF908B1012070BD64
:1042C000102C07D200222146501E00F07EF805482F
:1042D000046001E00120F2E70020F0E71400002074
:1042E000080000201000002010B510210248FFF740
:1042F00069FF0446204610BD0008014000B585B0A6
:1043000000BF1848806940F00800164988610846D7
:10431000806900F00800009000BF00BF00BF0846A1
:10432000806940F0010088610846806900F0010062
:10433000009000BF00BF00BF0B49486820F0E0605C
:1043400040F00070486000BF0120029003900320FD
:1043500004901020019001A90448FFF793FD05B0D7
:1043600000BD00000010024000000140000C0140B0
:1043700010B504462CB9012210210348FFF731FF84
:1043800000E000BF00BF10BD000C014010B50446A6
:1043900024B910210348FFF71DFF00E000BF00BF54
:1043A00010BD0000000C014070470146084600287F
:1043B00009DB00F01F0301229A4043099B0003F12F
:1043C000E023C3F8002100BF70472DE9F05F80466D
:1043D0000D461646002703F053FE074639462A4687
:1043E000334601F00700C0F1070ABAF1040F02D901
:1043F0004FF0040A01E0C0F1070AD14600F1040AB7
:10440000BAF1070F02D24FF0000A01E0A0F1030A4F
:10441000D4464FF0010A0AFA09FAAAF1010A0AEA97
:10442000020A0AFA0CFA4FF0010B0BFA0CFBABF183
:10443000010B0BEA030B4AEA0B042146404603F04A
:1044400027FEBDE8F09F000000BF00F00702064B0A
:1044500019684FF6FF031940044B0B4343EA02214E
:10446000014B196000BF70470CED00E00000FA0539
:104470002DE9F04385B0064642A30FCB01AC0FC433
:1044800044A0006800904FF0000800250027002499
:10449000A146042E36D004DC012E3BD0022E6BD177
:1044A0005FE0082E32D0102E66D13B484468006889
:1044B00000F0807000B301A8C4F38341475C04F4AA
:1044C000803070B134484068C0F340401DF800802F
:1044D00004F4803040B13148B0FBF8F000FB07F540
:1044E00002E02F4807FB00F52B48406800F48000ED
:1044F000B0F5800F01D1A94603E068000321B0FBAD
:10450000F1F93AE000F0D0F9814636E000F0CCF95C
:10451000814632E02048046A04F44070B0F5807FA0
:1045200005D104F0020010B14FF4004918E004F482
:104530004070B0F5007F07D11748406A00F00200D4
:1045400010B149F640490BE004F44070B0F5407FEB
:1045500006D11148006800F4003008B14FF2244938
:104560000BE000F091F90C494968C1F38131491C15
:104570004900B0FBF1F900E000BF00BF484605B0BC
:10458000BDE8F08302030405060708090A0B0C0DB9
:104590000E0F1010010200000010024000127A00FD
:1045A00000093D00F8B504460027002600252078C4
:1045B00000F00100002869D04248C06900F0805036
:1045C00070B900BF3F48C06940F080503D49C861A4
:1045D0000846C06900F08050009000BF00BF01276E
:1045E0003948006800F48070B0B93748006840F47A
:1045F000807035490860FFF7FBFD064606E0FFF7CF
:10460000F7FD801B642801D90320F8BD2E480068FF
:1046100000F480700028F2D02A48006A00F4407547
:104620002DB3A08800F44070A84220D02548006A2D
:1046300020F44075012025490860002008602148C9
:10464000056205F0010090B1FFF7D2FD064608E0D3
:10465000FFF7CEFD801B41F28831884201D903204B
:10466000D3E71848006A00F002000028F0D015488F
:10467000006A20F440706168084312490862012F03
:1046800004D10846C06920F08050C861207800F04D
:104690000200022807D10B48406820F44040A1687E
:1046A000084308494860207800F01000102807D11E
:1046B0000448406820F4800061690843014948606B
:1046C0000020A2E700100240007000404004424277
:1046D00070B504460D460CB9012070BD5A480068FB
:1046E00000F00700A8420ED25748006820F00700EB
:1046F0002843554908600846006800F00700A842B2
:1047000001D00120E9E7207800F0020002281DD145
:10471000207800F00400042805D14C48406840F49B
:10472000E0604A494860207800F00800082805D178
:104730004648406840F460504449486043484068F7
:1047400020F0F000A168084340494860207800F05C
:10475000010078B36068012806D13C48006800F485
:10476000003090B90120B8E76068022806D13748C8
:10477000006800F0007040B90120AEE733480068DF
:1047800000F0020008B90120A7E73048406820F097
:104790000300616808432D494860FFF729FD06467C
:1047A00009E0FFF725FD801B41F28831884202D9DC
:1047B000032092E707E02548406800F00C0061689C
:1047C000B0EB810FEDD12048006800F00700A8424F
:1047D0000ED91D48006820F0070028431A490860D8
:1047E0000846006800F00700A84201D0012074E7E5
:1047F000207800F00400042807D11448406820F411
:10480000E060E168084311494860207800F0080042
:10481000082808D10D48406820F46050216940EA1A
:10482000C1000A49486000F03FF808494968C1F3EF
:104830000311074A515CC8400649086006480068F1
:10484000FFF72CFD002048E7002002400010024046
:10485000B09C0008080000201000002001480068FB
:10486000704700000800002000B5FFF7F7FF04497B
:104870004968C1F30221034A515CC84000BD0000F1
:1048800000100240C09C000800B5FFF7E7FF044994
:104890004968C1F3C221034A515CC84000BD000011
:1048A00000100240C09C0008F0B585B00FF26C0CFF
:1048B0009CE8E01001A8A0E8E0101CA52D68009578
:1048C00000210022002300240020194D696801F016
:1048D0000C05F5B1042D02D0082D19D101E01548C1
:1048E00019E001ADC1F38346AC5D01F4803555B1EB
:1048F0000F4D6D68C5F340451DF805200D4D65430E
:10490000B5FBF2F302E00C4D04FB05F3184602E0A0
:1049100000BF084800BF00BF05B0F0BD020304059A
:10492000060708090A0B0C0D0E0F101001020000FB
:104930000010024000127A0000093D00F8B504465C
:104940000CB90120F8BD207800F00100002878D0D3
:10495000F848406800F00C0004280CD0F548406886
:1049600000F00C00082811D1F248406800F48030B3
:10497000B0F5803F0AD1EF48006800F4003000280D
:104980005FD0606800285CD10120DBE700BF606871
:10499000B0F5803F06D1E748006840F48030E54933
:1049A000086028E0606858B9E248006820F4803068
:1049B000E04908600846006820F4802008601AE09A
:1049C0006068B0F5A02F0BD1DA48006840F4802071
:1049D000D84908600846006840F4803008600AE062
:1049E000D448006820F48030D24908600846006846
:1049F00020F48020086000BF606888B1FFF7F8FBF2
:104A0000054606E0FFF7F4FB401B642801D90320AC
:104A100098E7C848006800F400300028F2D010E0A1
:104A2000FFF7E6FB054606E0FFF7E2FB401B6428C4
:104A300001D9032086E7BF48006800F40030002851
:104A4000F2D1207800F00200022857D1B94840681E
:104A500000F00C0050B1B748406800F00C00082886
:104A600018D1B448406800F4803098B9B148006863
:104A700000F0020020B12069012801D0012061E787
:104A8000AC48006820F0F800616940EAC100A9491B
:104A9000086033E02069E8B10120A7490860FFF70A
:104AA000A7FB054606E0FFF7A3FB401B022801D940
:104AB000032047E79F48006800F002000028F2D07A
:104AC0009C48006820F0F800616940EAC1009949FB
:104AD000086013E0002098490860FFF789FB05464D
:104AE00006E0FFF785FB401B022801D9032029E7D8
:104AF0009048006800F002000028F2D1207800F011
:104B0000080008282DD1A069B8B101208B490860A0
:104B1000FFF76EFB054606E0FFF76AFB401B022825
:104B200001D903200EE78348406A00F00200002804
:104B3000F2D0012002F00AFD13E000207F49086056
:104B4000FFF756FB054606E0FFF752FB401B022825
:104B500001D90320F6E67748406A00F002000028F9
:104B6000F2D1207800F00400042873D100277148A6
:104B7000C06900F0805070B900BF6E48C06940F055
:104B800080506C49C8610846C06900F080500090B0
:104B900000BF00BF01276A48006800F48070B0B908
:104BA0006748006840F4807065490860FFF720FBA3
:104BB000054606E0FFF71CFB401B642801D90320D3
:104BC000C0E65F48006800F480700028F2D000BFA3
:104BD000E068012806D15748006A40F001005549B5
:104BE000086227E0E06858B95248006A20F00100E6
:104BF000504908620846006A20F00400086219E083
:104C0000E06805280BD14B48006A40F00400494990
:104C100008620846006A40F0010008620AE0454860
:104C2000006A20F00100434908620846006A20F04B
:104C30000400086200BFE068A0B1FFF7D9FA05469A
:104C400009E0FFF7D5FA401B41F28831884202D9CA
:104C5000032077E622E03748006A00F002000028CF
:104C6000EFD012E0FFF7C4FA054608E0FFF7C0FAFC
:104C7000401B41F28831884201D9032062E62D4869
:104C8000006A00F002000028F0D1012F05D1294868
:104C9000C06920F080502749C86100BFE069C8B3EF
:104CA0002448406800F00C00082860D0E069022821
:104CB00048D1002020490866FFF79AFA054606E029
:104CC000FFF796FA401B022801D903203AE619485B
:104CD000006800F000700028F2D1206AB0F5803F33
:104CE00007D11448406820F40030A16808431149F6
:104CF0004860D4E9080108430E49496821F4741159
:104D000008430C49486001200B490866FFF770FA18
:104D1000054607E03DE0FFF76BFA401B022801D98A
:104D200003200FE60348006800F000700028F2D06E
:104D30002FE0000000100240000042428004424286
:104D400000700040002014490866FFF751FA05463C
:104D500006E0FFF74DFA401B022801D90320F1E5D8
:104D60000E48006800F000700028F2D111E0E06900
:104D7000012800D1E6E50948466806F48031206A3A
:104D8000814204D106F47011606A814201D0012091
:104D9000D8E50020D6E500000000424200100240A5
:104DA00010B504460CB9012010BD022084F8510052
:104DB0002068006820F0400021680860204600F06C
:104DC00058F80020606584F8510000BF84F8500056
:104DD00000BF00BFE8E710B504460CB9012010BDC4
:104DE000606A00B900BFA06AB0F5005F00D100BFE3
:104DF00094F8510028B9002084F85000204600F0B3
:104E000039F8022084F851002068006820F0400042
:104E100021680860D4E901010843E1680843216979
:104E2000084361690843218B01F400710843E1697B
:104E30000843216A0843A16A0843216808600421E5
:104E4000A06901EA104021684860A06AB0F5005FDF
:104E500002D12168E06A08612068C06920F400601E
:104E60002168C86100206065012084F8510000209D
:104E7000B5E7704710B586B0044600BF1348806997
:104E800040F00400114988610846806900F0040080
:104E9000019000BF00BF00BF0846806940F4805009
:104EA00088610846806900F48050019000BF00BF0F
:104EB000E02002900220039000200490032005903F
:104EC00002A90348FEF7DEFF06B010BD0010024045
:104ED000000801402DE9F8430446884617461D4660
:104EE0004FF000096068B0F5827F0DD1A06858B915
:104EF000042084F851003B46424641462046009536
:104F000000F0FAF9BDE8F88300BF94F850000128DA
:104F100001D10220F6E7012084F8500000BFFFF71E
:104F200067F9064694F85100012802D04FF00209B3
:104F3000EBE0B8F1000F00D017B94FF00109E4E041
:104F4000042084F8510000206065C4F83880A787E9
:104F5000E7872063A086E08620646064A06AB0F5DD
:104F6000005F10D100BF2068006820F40050216865
:104F700008602068006840F400502168086000BFA5
:104F8000E08F401EE087A068B0F5004F05D1206893
:104F9000006820F48040216808602068006800F004
:104FA0004000402805D02068006840F0400021689B
:104FB0000860E068F8B91AE02068806800F0010035
:104FC00050B12068007BA16B0870A06B401CA063EF
:104FD000E08F401EE0870AE0FFF70AF9801BA84235
:104FE00001D3681C00B915B94FF003098DE0E08FBB
:104FF0000028E1D11EE01AE02068806800F001007E
:1050000050B12068C068A16B0880A06B801CA063B1
:10501000E08F401EE0870AE0FFF7EAF8801BA84215
:1050200001D3681C00B915B94FF003096DE0E08F9A
:105030000028E1D1A06AB0F5005F39D1206800688E
:1050400040F48050216808602068006800F48050B7
:1050500028B12068006820F48050216808602B4641
:10506000012211462046009602F099FB10B14FF044
:1050700003094AE0E068B0F5006F04D12068C06819
:10508000A16B088003E02068007BA16B08702B46B1
:10509000012211462046009602F081FB30B1606D7E
:1050A00040F0020060654FF003092EE02068C06800
:1050B00032462946204602F01FFB08B120206065D9
:1050C00020688068C0F30010D0B1204602F064FB75
:1050D000012811D1606D40F00200606500BF2068BA
:1050E000006820F40050216808602068006840F4DF
:1050F00000502168086003E04FF6EF702168886077
:10510000606D08B14FF0010900BF012084F8510023
:1051100000BF002084F8500000BF4846F2E62DE9A9
:10512000F84F0446884616461D464FF0000A00BF59
:1051300094F85000012802D10220BDE8F88F012028
:1051400084F8500000BFFFF753F80746B14694F8C3
:105150005100012802D04FF0020AC3E0B8F1000F5D
:1051600000D016B94FF0010ABCE0032084F85100CA
:1051700000206065C4F83080A686E686A063A0871C
:10518000E08760642064A068B0F5004F05D1206816
:10519000006840F4804021680860A06AB0F5005FB4
:1051A0000DD100BF2068006820F40050216808601D
:1051B0002068006840F400502168086000BF206843
:1051C000006800F04000402805D02068006840F0EA
:1051D000400021680860E068B0F5006F2FD160687A
:1051E00010B1B9F1010F09D1206B00882168C860A6
:1051F000206B801C2063E08E401EE0861BE0206850
:10520000806800F0020002280AD1206B0088216823
:10521000C860206B801C2063E08E401EE0860AE0A0
:10522000FEF7E6FFC01BA84201D3681C00B915B900
:105230004FF0030A56E0E08E0028E0D12EE06068CF
:1052400010B1B9F1010F09D1206B00782168087302
:10525000206B401C2063E08E401EE0861BE020682F
:10526000806800F0020002280AD1206B00782168D3
:105270000873206B401C2063E08E401EE0860AE02D
:10528000FEF7B6FFC01BA84201D3681C00B915B9D0
:105290004FF0030A26E0E08E0028E0D1A06AB0F5C6
:1052A000005F05D12068006840F4805021680860E4
:1052B0003A462946204602F05BFA08B12020606594
:1052C000A06850B900BF002000902068C06800901E
:1052D00020688068009000BF00BF606D08B14FF08B
:1052E000010A00BF012084F8510000BF002084F8AB
:1052F000500000BF504620E72DE9FF5F0446884676
:1053000091461D460E9E012002900020019000BF94
:1053100094F85000012803D1022004B0BDE8F09FAA
:10532000012084F8500000BFFEF762FF074694F8A2
:1053300051B060680390AA46BBF1010F0BD00398EF
:10534000B0F5827F04D1A06810B9BBF1040F02D080
:10535000022001903DE1B8F1000F03D0B9F1000F38
:1053600000D015B90120019033E194F851000428D0
:1053700002D0052084F8510000206065C4F8389000
:10538000E587A587C4F83080E586A586206460643B
:10539000A06AB0F5005F0DD100BF2068006820F45E
:1053A0000050216808602068006840F400502168BF
:1053B000086000BF2068006800F04000402805D069
:1053C0002068006840F0400021680860E068B0F59F
:1053D000006F56D1606810B1BAF1010F09D1206B8E
:1053E00000882168C860206B801C2063E08E401E0E
:1053F000E0863FE02068806800F0020002281CD1AF
:10540000E08ED0B10298012817D1206B0088216866
:10541000C860206B801C2063E08E401EE086002068
:105420000290E08E48B9A06AB0F5005F05D120680F
:10543000006840F48050216808602068806800F0AF
:10544000010068B1E08F58B12068C068A16B088086
:10545000A06B801CA063E08F401EE08701200290BB
:10546000FEF7C6FEC01BB04204D3701C10B103206F
:105470000190AEE0E08E0028BCD1E08F0028B9D1C9
:1054800056E0606810B1BAF1010F09D1206B0078C5
:1054900021680873206B401C2063E08E401EE0866C
:1054A00040E02068806800F0020002281CD1E08EF5
:1054B000D0B10298012817D1206B007821680873B9
:1054C000206B401C2063E08E401EE086002002908E
:1054D000E08E48B9A06AB0F5005F05D12068006889
:1054E00040F48050216808602068806800F0010066
:1054F00068B1E08F58B12068C068A16B0870A06BDC
:10550000401CA063E08F401EE08701200290FEF760
:105510006FFEC01BB04201D3701C00B916B9032046
:10552000019056E0E08E0028BBD1E08F0028B8D172
:10553000A06AB0F5005F10D1334601221146204623
:10554000009702F02CF930B1606D40F00200606508
:10555000032001903DE02068C06820688068C0F3A7
:105560000010E8B1204602F017F9012814D1606D4F
:1055700040F00200606500BF2068006820F4005021
:10558000216808602068006840F4005021680860C5
:1055900000BF0120019003E04FF6EF7021688860A2
:1055A0003A463146204602F0E3F820B1012001904E
:1055B000202060650DE0A06850B900BF0020009079
:1055C0002068C068009020688068009000BF00BF1D
:1055D00000BF012084F8510000BF002084F8500073
:1055E00000BF019899E6042808D14FF0E02109692D
:1055F00041F004014FF0E022116107E04FF0E0219B
:10560000096921F004014FF0E0221161704770B583
:1056100004462546681EB0F1807F01D301200FE0CB
:10562000681E4FF0E02148610F214FF0FF3002F07B
:105630002FFD00204FF0E021886107200861002045
:1056400070BD000000B585B000BF0D48806940F016
:1056500004000B4988610846806900F0040000904E
:1056600000BF00BF20200190002002900120039085
:105670000320049001A90348FEF704FC05B000BD17
:10568000001002400008014010B501F0C5FF2820BD
:1056900001F0FCFF10BD000010B504460448046092
:1056A00001F068FF01F08EFFFFF7EEFF10BD000074
:1056B0004400002070B504460D460026002000F08E
:1056C0000BF82946204601F0CFFF0646012000F0E6
:1056D00003F8304670BD000010B504462CB101221D
:1056E00004210548FEF77DFD04E000220421024864
:1056F000FEF777FD10BD00000008014070B50446BC
:105700000D4600260020FFF7E7FF2946204601F05E
:10571000E1FF06460120FFF7DFFF304670BD0000C5
:1057200010B50248FFF73CFB10BD0000444C0020C0
:105730000FB438B5044606A8009080212046009B8F
:10574000059AFAF7EDFD054600200090284638BC82
:105750005DF814FB10B5FEF74BFD10BD70477047A8
:1057600010B504460CB9012010BD94F83D0028B9CD
:10577000002084F83C00204600F00CF8022084F859
:105780003D00211D206802F0E3F9012084F83D006E
:105790000020E9E738B504460D492068884215D154
:1057A00000BF0C48C06940F002000A49C8610846C1
:1057B000C06900F00200009000BF00BF0322012179
:1057C0001D20FEF702FE1D20FEF7EFFD38BD000094
:1057D000000400400010024001460868C06840F024
:1057E00001000B68D8600868806800F00702062A8C
:1057F00005D00868006840F001000B6818600020C0
:105800007047704710B5044620680069C0F3400037
:10581000D8B12068C068C0F34000B0B16FF002009A
:1058200021680861012020772068806900F003006A
:1058300018B12046FFF7E5FF05E0204600F0ADF87F
:10584000204600F0ABF80020207720680069C0F304
:105850008000D8B12068C068C0F38000B0B16FF09C
:10586000040021680861022020772068806900F424
:10587000407018B12046FFF7C4FF05E0204600F055
:105880008CF8204600F08AF8002020772068006914
:10589000C0F3C000D8B12068C068C0F3C000B0B188
:1058A0006FF0080021680861042020772068C06933
:1058B00000F0030018B12046FFF7A3FF05E02046E3
:1058C00000F06BF8204600F069F80020207720688F
:1058D0000069C0F30010D8B12068C068C0F30010A0
:1058E000B0B16FF0100021680861082020772068AF
:1058F000C06900F4407018B12046FFF782FF05E050
:10590000204600F04AF8204600F048F800202077B2
:105910002068006900F0010058B12068C06800F0FC
:10592000010030B16FF0010021680861204600F0ED
:1059300037F820680069C0F3C01058B12068C0680B
:10594000C0F3C01030B16FF08000216808612046BC
:10595000FFF704FF20680069C0F3801058B1206889
:10596000C068C0F3801030B16FF04000216808615A
:10597000204600F01FF820680069C0F3401058B1BD
:105980002068C068C0F3401030B16FF0200021687B
:1059900008612046FFF7E3FE10BD70477047000026
:1059A00010B504460248844201D100F057F810BDFA
:1059B000044C00207047000070B505460C460748AF
:1059C000074908600846446000218160C5600161A4
:1059D000FFF7C6FE0248FFF7FFFE70BD000400405F
:1059E000044C002030B502460B460020002111E097
:1059F000194C04EB0114246894420AD1164C04EBB0
:105A00000114A3600024144D05EB0115EC60C8B22D
:105A100030BD491C2029EBDB002118E00E4C04EBC3
:105A20000114246894B90C4C04EB011422600A4D53
:105A300005EB01152971084C04EB0114A360002447
:105A4000054D05EB0115EC60C8B202E0491C2029A8
:105A5000E4DB00BF00BFDBE79459002010B5002451
:105A60001EE0114800EB04100068C0B10E4800EBC6
:105A70000410C068401C0C4901EB0411C8600A49BD
:105A800001EB04118968884209DB0020064901EB1B
:105A90000411C860044901EB041108688047641CC4
:105AA000202CDEDB10BD0000945900207047014619
:105AB0000022002391F8392091F83A3042EA03009D
:105AC000704700002DE9F04704462068056820680B
:105AD000C668206847694FF00008C14605F00F0806
:105AE000B8F1000F0AD105F0200038B106F020000F
:105AF00020B1204602F0A4F8BDE8F087B8F1000F0D
:105B00006DD007F0010018B906F49070002866D037
:105B100005F0010030B106F4807018B1E06B40F080
:105B20000100E06305F0040030B107F0010018B196
:105B3000E06B40F00200E06305F0020030B107F0D6
:105B4000010018B1E06B40F00400E06305F00800CC
:105B500030B107F0010018B1E06B40F00800E063DD
:105B6000E06B68B305F0200028B106F0200010B10A
:105B7000204602F065F820684069C0F38019E06BA8
:105B800000F0080010B9B9F1000F22D0204602F051
:105B900037F82068406900F04000B0B120684069E3
:105BA00020F0400021684861606B50B11748616B7C
:105BB0004863606BFDF754FF10B1606B416B884721
:105BC0000CE02046FFF772FF08E02046FFF76EFF6B
:105BD00004E02046FFF76AFF0020E0638CE705F051
:105BE000800030B106F0800018B1204602F04CF978
:105BF00082E705F0400030B106F0400018B12046C1
:105C000002F00EF878E700BF76E70000ED7B0008B1
:105C100010B504460CB9012010BDA06900B100E028
:105C200000BF94F8390028B9002084F838002046D5
:105C300000F028F8242084F839002068C06820F497
:105C400000502168C860204602F04EF820680069C4
:105C500020F49040216808612068406920F02A0003
:105C6000216848612068C06840F400502168C8601D
:105C70000020E063202084F8390084F83A000020F6
:105C8000CAE7000010B586B004462549206888425E
:105C900044D100BF2348806940F004002149886155
:105CA0000846806900F00400019000BF00BF00BFFB
:105CB0000846806940F4804088610846806900F4A5
:105CC0008040019000BF00BF00BF0846806940F0DF
:105CD000010088610846806900F00100019000BF62
:105CE00000BF481502900220039001200490032079
:105CF000059002A90C48FEF7C5F84FF480600290A9
:105D00000020039002A90848FEF7BCF82520FEF702
:105D10004CFB032211462520FEF757FB06B010BDB1
:105D200000380140001002400008014010B5034651
:105D300093F83A0020282FD101B10AB9012010BDF3
:105D400000BF93F83800012801D10220F7E70120B5
:105D500083F8380000BF99629A85DA850020D863FD
:105D6000222083F83A0000BF002083F8380000BFEB
:105D70001868C06840F480701C68E060186840696A
:105D800040F001001C6860611868C06840F02000A5
:105D90001C68E0600020D2E70220D0E710B504467E
:105DA00022492068884240D12148008800F4004000
:105DB00000283AD11E48008800F48040B8B11D4840
:105DC00000780A2803D00020194908802DE01848DF
:105DD000008840F4004016490880084601781648BB
:105DE000164A126890470020114908801DE01148AA
:105DF00000780D2806D10E48008840F480400C49F8
:105E0000088012E00B48007809490988C1F30D01A8
:105E1000094A505406480088401C05490880084635
:105E20000088C72801DD0020088010BD003801402F
:105E30002000002022000020A04A00202400002092
:105E40002DE9F84304460D4616461F464FF000095B
:105E500094F8390020285CD105B116B90120BDE8BD
:105E6000F88300BF94F83800012801D10220F6E73A
:105E7000012084F8380000BF0020E063212084F86E
:105E80003900FEF7B5F98146A684E6842BE0E08C64
:105E9000401EE084A068B0F5805F16D14B4600221A
:105EA00080212046009702F023F808B10320D6E7AE
:105EB000A846B8F80000C0F30800216848602069CF
:105EC00008B9AD1C0FE06D1C0DE04B46002280218F
:105ED0002046009702F00CF808B10320BFE715F840
:105EE000010B21684860E08C0028D0D14B4600228D
:105EF00040212046009701F0FBFF08B10320AEE7E8
:105F0000202084F8390000BF002084F8380000BF4A
:105F1000A5E70220A3E77047014908607047000029
:105F20002400002070B504460D464FF47A732A46CB
:105F300021460248FFF784FF70BD0000684B002037
:105F40007FB504460D461646324629462046039B39
:105F5000FAF7E6F904B070BD10B54FF47A71024853
:105F6000FFF740FD10BD0000B999000870B5044668
:105F70000D46044804490860084644608560FEF701
:105F80003DF970BD00300040CC4C002000BFFEE762
:105F90002DE9F04F91B08246894600242021F8482F
:105FA000FAF70EFD4A465146F548FAF750FCF44C14
:105FB0000822F4A12046FAF7F3FBA0B940F2F165FC
:105FC000F3A103C9CDE90F012C21F3A0FCF714FACA
:105FD00010B1F7A002F026F808230FAA29460020E6
:105FE000FDF7A8FC70E30822F6A12046FAF7D8FBDB
:105FF000002813D140F2F1653422F5A104A8FAF784
:10600000ADFC3C21E4A0FCF7F7F910B1FDA002F0D3
:1060100009F8342104A800F085FC55E30922FCA10D
:106020002046FAF7BDFB10B901F056FD4CE30822FB
:10603000FAA12046FAF7B4FBA8B9002504E005F15F
:10604000F10009A948556D1C202DF8DB4B21D2A089
:10605000FCF7D2F910B1F4A001F0E4FF202109A867
:10606000FFF74CFB30E30922F3A12046FAF798FB37
:1060700060B902F01FF905465121C7A0FCF7BCF931
:1060800018B12946EFA001F0CDFF1DE30C22F1A1CC
:106090002046FAF785FB28B900221146062000F0B9
:1060A000ADFD11E30922EFA12046FAF779FB60B9B3
:1060B000FEF71AF905465A21B7A0FCF79DF918B169
:1060C0002946EBA001F0AEFFFEE20922ECA120463A
:1060D000FAF766FB20BBFCF7BDFD1090109803F0AB
:1060E000CEFC4FF06632E94BCDE90C0103F0DEFC4B
:1060F00007460022E64B03F0D9FC054603F090FC6E
:1061000083460BEB4B0040000F906221A2A0FCF7EE
:1061100073F920B1DFA0DDE90F2101F083FFD3E2A5
:106120000B22E3A12046FAF73BFB48B9E3A207CADA
:106130000EAB07C309220EA9032000F05FFDC3E2E6
:106140000822E1A12046FAF72BFB28B9FFF79CFAB9
:106150000120FCF7DFFDB7E20922DEA12046FAF7B5
:106160001FFB28B90020FCF7D5FDFFF76BFAABE267
:106170000C22DBA12046FAF713FB50B9752186A04B
:10618000FCF73AF910B1DAA001F04CFFFCF7D4FDAE
:106190009AE20F22D9A12046FAF702FBC8B904F10E
:1061A0000F00FAF793FAC5B27B217BA0FCF724F924
:1061B00018B12946D5A001F035FF012D03D1D748EC
:1061C00000F0D2FE04E0022D02D1D54800F0CCFE52
:1061D0007AE20A22D3A12046FAF7E2FAC8B904F11A
:1061E0000A00FAF773FAC5B289216BA0FCF704F92B
:1061F00018B12946C5A001F015FF012D03D1C748EC
:10620000FDF7E2FD04E0022D02D1C548FDF7DCFDFB
:106210005AE20A22C6A12046FAF7C2FA00282FD174
:1062200004F10A00FAF752FAC6B29A215AA0FCF712
:10623000E3F818B13146C1A001F0F4FE002502E0F8
:1062400001A94D556D1C402DFADB012E06D14022CF
:1062500001A9B248FDF7BEFD074607E0022E05D1B1
:10626000402201A9AE48FDF7B5FD0746A9214AA085
:10627000FCF7C2F818B13946B4A001F0D3FE23E20E
:106280000922B7A12046FAF78BFA00283DD1B021A8
:1062900041A0FCF7B1F818B12946B4A001F0C2FE44
:1062A000402101A8FAF7AEFB04F10900FAF70EFA53
:1062B000C5B2012D13D1402201A99848FDF779FDFF
:1062C000B92135A0FCF798F8F0B1402101A801F000
:1062D000BBFA06463146A9A001F0A4FE14E0022D47
:1062E00012D1402201A98E48FDF763FDBE212AA0EC
:1062F000FCF782F840B1402101A801F0A5FA06465A
:1063000031469EA001F08EFEDEE10B229FA12046C9
:10631000FAF746FA50B9C3211FA0FCF76DF810B187
:106320009DA001F07FFE01F053F8CDE107229DA171
:106330002046FAF735FA00BB00200F901090E07964
:106340003F281CD1002000F0B5FE01680F91808825
:10635000ADF84000CE2110A0FCF74EF870B19DF8CA
:1063600041009DF840109DF83F20CDE900210290AA
:106370009DF83E309DF83D2018E137E135E11BE105
:10638000D84C002041542B43414E5458000000008B
:10639000600322F18BFFFFFF2E2E5C4D4F445C53B8
:1063A00072635C6D6F645F6174636D642E63000083
:1063B00073656E64206461746120746F2063616E24
:1063C0000000000041542B49534F54580000000076
:1063D00062F101010100042106228F04D2010000B4
:1063E000100000000100003CFB0400000600003C1F
:1063F000FC04000008000034EC0D0000080000431D
:106400004E0D000169736F313537363520747800D1
:1064100041542B5245424F4F5400000041542B53DE
:1064200050495458000000007370692073656E6411
:10643000206461746100000041542B4D4355564562
:1064400052000000736F66745F7665723A3078258B
:106450007800000041542B474554424C4556455264
:106460000000000041542B4B45595354410000009B
:106470006B6579207374617475733A25640000004C
:1064800041542B41444356414C00000066664A3F4C
:1064900000408F406164765F76616C3A25642C62BF
:1064A0006174746572795F6D763A25646D7600006B
:1064B00041542B5350495452414E53005212000044
:1064C0000006F1011100000041542B424C454F4E93
:1064D0000000000041542B424C454F46460000004E
:1064E00041542B424C455245424F4F54000000004E
:1064F0007265626F6F7420626C65000041542B43BB
:106500004845434B534543544F523D0065726173B8
:10651000655F696E6465783A2564000000F40308DD
:1065200000F0030841542B4645524153453D0000BD
:1065300041542B4657524954453D000077726974C7
:10654000655F696E6465783A2564000077726974E6
:106550006520666C617368207265743A256400007A
:1065600041542B46524541443D0000007265616430
:106570005F696E6465783A25640000007265616445
:106580005F746D705F6275663A25730041542B53DA
:10659000484F57504152410073686F7720706172C5
:1065A0006100000041542B4D41433D009DF83C10DB
:1065B00047A001F037FD18E0A9F107000C280AD028
:1065C000D421AFF22C20FBF717FF20B1A9F107016E
:1065D00045A001F027FD0C21E01D01F061F9054601
:1065E0002A460621002000F067FE6DE0082244A143
:1065F0002046FAF7D5F8B8BB00200F901090002580
:106600000026207A3F2813D1012000F053FD0646D2
:10661000E221AFF27C20FBF7EFFE20B33046FAF721
:10662000A0F807463A46314638A001F0FBFC1AE0D4
:10663000A9F10800C5B22A4604F108010FA8FAF72B
:1066400006F900200FA94855EA21AFF2B420FBF764
:10665000D3FE18B10FA932A001F0E4FC0FAA29461D
:10666000012000F029FE2FE0FFE70C2230A1204698
:10667000FAF796F840BB00201090207B3F280ED1FF
:10668000F321AFF2EC20FBF7B7FEE0B1022000F0FF
:1066900011FD056829462AA001F0C4FC13E004F1AD
:1066A0000C00FAF713F81090F821AFF21430FBF752
:1066B000A3FE18B128A0109901F0B4FC10AA04217F
:1066C000022000F0F9FD00BF11B0BDE8F08F00001E
:1066D000626C655F6D61633A2558255825582558C9
:1066E0002558255800000000696E707574206D6192
:1066F00063206C656E3A2564206572726F720000CB
:1067000041542B4E414D453D00000000626C655FD9
:106710006E616D653A25732C6C656E3A25640000D8
:1067200073657420626C655F6E616D653A257300F8
:1067300041542B494E54455256414C3D00000000F7
:10674000626C655F6164765F696E74657276616CB8
:106750003A25646D7300000073657420626C655F98
:10676000696E74657276616C3A25640010B5002418
:1067700006E0054901EBC401486801F06DFE641CA8
:10678000042CF6D310BD00001026002070B50025A3
:1067900000240BE0074901EBC401486801F004FE46
:1067A000054615B14FF0FF3070BD641C042CF1D3C9
:1067B0000020F9E7102600202DE9F04186B00546BB
:1067C0008846D5F8016001960120ADF80C00042040
:1067D00002906879ADF80E00002004900590BDF895
:1067E0000E20A91D04A8FAF732F8D22128A0FBF741
:1067F00003FE60B1BDF80E1004A801F025F80446B0
:10680000BDF80E202346314629A001F00BFC0027DD
:10681000002416E0364850F83400019988420FD120
:10682000DE211BA0FBF7E8FD10B132A001F0FAFB5E
:1068300001272F4901EBC401486801A901F0A7FD18
:10684000641C042CE6D3002F1FD100241AE0284832
:1068500050F83400B0F1FF3F13D1EA210CA0FBF750
:10686000CBFD18B1214627A001F0DCFB204901989F
:1068700041F8340001EBC401486801A901F087FD2B
:1068800002E0641C042CE2D300BF06B0BDE8F08136
:106890002E2E5C4D4F445C5372635C6D6F645F637E
:1068A000616E6461746170726F636573732E6300EF
:1068B0007075742063616E20746F20313537363502
:1068C0002070617273652C63616E5F69643A307821
:1068D00025782C7061796C6F61645F6C656E3A2508
:1068E000642C7061796C6F61643A2573000000005C
:1068F0001026002066696E64206672616D655F69AE
:10690000640000006E6F742066696E6420667261B8
:106910006D655F69642C206E6F7720736574202528
:106920006400000070B504460D46B5F5017F02DD38
:106930004FF4017000E028461749C8814FF40171F7
:1069400015481030FAF73CF81348C2892146103038
:10695000F9F77DFF06201049487012210E4881701A
:10696000DF21C1700021017140F219110BA0FBF76A
:1069700043FD58B10848C189103000F065FF064654
:106980000548C18932460DA001F04CFB024916486A
:1069900001F04FFF70BD00004A0000202E2E5C4D1C
:1069A0004F445C5372635C6D6F645F63616E6461DE
:1069B000746170726F636573732E630073656E64C8
:1069C0002063616E206461746120746F2069736F4D
:1069D00031353736352C73697A653A25642C646114
:1069E00074613A2553000000600200202DE9FE4F3B
:1069F00004460F4626464FF0000A4FF0040B0020D5
:106A00000190F57896F80280ABF102004044C01E78
:106A100000F0FF094946A01C01F0D0FA824609F1B6
:106A2000020020440088029002A802F075FFBDF821
:106A30000800824501D0BDE8FE8F2E213DA0FBF766
:106A4000DBFC48B13946204600F0FEFE3A460146DE
:106A500000903EA001F0E6FA012D15D120790190B9
:106A6000332134A0FBF7C8FC10B13EA001F0DAFAE4
:106A7000342130A0FBF7C0FC18B13DA0019901F012
:106A8000D1FA00F02BF953E0072D09D1392129A0C3
:106A9000FBF7B2FC00284BD039A001F0C3FA47E065
:106AA000032D19D13D2123A0FBF7A6FC10B137A07F
:106AB00001F0B8FA207951283AD140211DA0FBF706
:106AC0009BFC10B136A001F0ADFAA8F10400C1B2F0
:106AD000601DFFF727FF2BE0042D09D1462115A0EB
:106AE000FBF78AFC002823D032A001F09BFA1FE0BC
:106AF000052D08D14A210FA0FBF77EFCC0B131A0C3
:106B000001F090FA14E0062D12D1207901904F2166
:106B100008A0FBF771FC10B12FA001F083FA5021FF
:106B200004A0FBF769FC18B12FA0019901F07AFAD3
:106B300000BF80E72E2E5C4D4F445C5372635C6D4A
:106B40006F645F7370692E63000000007370695F8B
:106B500072785F646174613A25732C6C656E3A25B6
:106B600064000000424C455F434D445F564552006F
:106B7000626C65207665723A3078257800000000F6
:106B8000424C455F434D445F43464700424C455F9E
:106B9000434D445F5452414E53464552000000005D
:106BA00073656E645F63616E5F646174615F636D82
:106BB00064000000424C455F434D445F434F4E4EDE
:106BC00045435400424C455F434D445F4449534361
:106BD0004F4E4E4543540000424C455F434D445F89
:106BE000544553540000000067657420626C6520B2
:106BF0007665723A30782578000000002DE9F04F74
:106C000091B080468A461446402101A8F9F7FAFE61
:106C10004FF00009042501AE402101A8F9F7F2FE6A
:106C2000F12030707070E01CB07086F80380002C8A
:106C300009DDC5F13E00A04205DD01A94819224643
:106C40005146F9F704FEA81E01190DF1060001F0E6
:106C5000B5F90746380A291901AA50542819401CC9
:106C60001754281900F1020973210CA0FBF7C4FB8B
:106C700048B1494601A800F0E7FD83464A46594617
:106C80000CA001F0CFF91148006820B1402101A803
:106C90000E4A1268904711B0BDE8F08F2E2E5C4D61
:106CA0004F445C5372635C6D6F645F7370692E63F5
:106CB000000000007370695F74785F646174613A0A
:106CC00025732C6C656E3A25640000003426002084
:106CD00001490860704700003426002070B58AB072
:106CE00000200890099005900690079004900024D9
:106CF00000250890099000F0DDF90168089180886E
:106D0000ADF82400852130A0FBF776FB88B19DF813
:106D100025009DF824109DF82320CDE90021029044
:106D20009DF822309DF821209DF820102CA001F024
:106D300079F90020059006900790012000F0BAF93B
:106D400004462046F9F70DFDC5B22A46214605A89E
:106D5000F9F77DFD8C211CA0FBF74EFB20B12A46E4
:106D600005A926A001F05EF9022000F0A3F9006851
:106D700004908F2114A0FBF73FFB18B125A00499C4
:106D800001F050F92021294800F058F808AB0622FC
:106D90000121264800F064F805AB2A460221234869
:106DA00000F05EF804AB04220321204800F058F8FC
:106DB00000F03EF8C6B232461C490720FFF71EFF1E
:106DC00000200AB070BD00002E2E5C4D4F445C5375
:106DD00072635C6D6F645F7370692E630000000006
:106DE00073657420626C655F6D61633A2558255840
:106DF0002558255825582558000000007365742033
:106E0000626C655F6E616D653A25732C6C656E3AD8
:106E10002564000073657420626C655F6164765F51
:106E2000696E74657276616C3A256400F84C0020D6
:106E300001480088704700003226002070B50546E2
:106E40000C46054804800020044908802146284655
:106E5000F9F7B6FD70BD0000302600203226002074
:106E60002DE9F04104460E4615461F461F4800888E
:106E70002844001D1E49098888420DDDCD211DA032
:106E8000FBF7BAFA30B1194800882844011D1FA049
:106E900001F0AEF8BDE8F081310A1448028800889C
:106EA000401C124B1880A154184602880088401CD0
:106EB0001880A654290A184602880088401C1880A9
:106EC000A154184602880088401C1880A554194611
:106ED000098860182A463946F9F7B9FC0348008842
:106EE00028440249088000BFD4E700003226002071
:106EF000302600202E2E5C4D4F445C5372635C6D37
:106F00006F645F7370692E6300000000746C7620FC
:106F100062756666657220697320746F6F20736D89
:106F2000616C6C5B25645D0010B502460023032490
:106F300013E0181941100B4810F83100904202DD9F
:106F4000481E84B209E0074810F83100904202DA86
:106F5000481C83B201E008B210BDA342E9DD4FF046
:106F6000FF30F9E7E09C000838B5054600240BE047
:106F7000042101FB04500A46694600F064F80098B9
:106F8000401C00B102E0641CFF2CF1DD00BFFF2CAF
:106F900009DC482109A0FBF72FFA10B10DA001F080
:106FA00041F8012038BD4B2104A0FBF725FA10B1B0
:106FB0000CA001F037F80020F4E700002E2E5C4D05
:106FC0004F445C5372635C6D6F645F7379732E63BF
:106FD0000000000074686572652069732064617444
:106FE00061000000736563746F7220656D70747961
:106FF0000000000010B50446342106A0FBF7FCF9A0
:1070000018B1214609A001F00DF82046FCF7DCFE7E
:1070100010BD00002E2E5C4D4F445C5372635C6DBE
:107020006F645F7379732E63000000006572617393
:107030006520616464723A307825780010B50020CC
:10704000FCF7B4FE10BD70B504460D461646324638
:1070500029462046FCF7ADFE70BD000070B5044621
:107060000D461646292107A0FBF7C6F920B1324686
:1070700021460AA000F0D6FF324629462046FCF7FA
:10708000A9FE70BD2E2E5C4D4F445C5372635C6D47
:107090006F645F7379732E63000000007772697408
:1070A0006520616464723A307825782C206C656EB6
:1070B0003A25640070B505462846FFF735FF0446BB
:1070C000B4F1FF3F09D1E02106A0FBF795F910B11B
:1070D0000AA000F08DFF002070BD0B4800EBC4003B
:1070E0004068F9E72E2E5C4D4F445C5372635C6D33
:1070F0006F645F7379732E630000000070617261CA
:107100002045727200000000E09C000810B5FFF7F7
:1071100095FF00F001F810BD10B58CB000241822C6
:1071200006A94548FCF745FE00281BD116210DF1A4
:107130001A0000F043FFBDF8181088420AD18421DC
:107140003EA0FBF759F910B142A000F06BFF44F0EC
:10715000010407E0892139A0FBF74EF910B141A0E5
:1071600000F060FF182269464348FCF722FE002821
:107170001BD116210DF1020000F020FFBDF8001018
:1071800088420AD191212DA0FBF736F910B13BA01E
:1071900000F048FF44F0020407E0962127A0FBF727
:1071A0002BF910B139A000F03DFF6CB918213C4813
:1071B000F9F728FC18223B493948F9F7CFFB182189
:1071C000374800F083F934E0012C11D1182206A9C8
:1071D0003348F9F7C3FB2848FFF7C6FE10B126482D
:1071E000FFF708FF18222E492348FFF737FF20E05A
:1071F000022C11D1182269462948F9F7AFFB0E4835
:10720000FFF7B2FE10B10C48FFF7F4FE1822244934
:107210000948FFF723FF0CE0182206A92048F9F7D8
:107220009DFBB62105A0FBF7E7F810B11EA000F00A
:10723000F9FE0CB010BD000000F403082E2E5C4DCA
:107240004F445C5372635C6D6F645F7379732E633C
:10725000000000006D61696E2070617261206F6BCB
:10726000000000006D61696E2070617261206E6FB8
:1072700074206F6B0000000000F003086261636B14
:1072800075702070617261206F6B00006261636BCA
:1072900075702070617261206E6F74206F6B0000DA
:1072A000184D0020C89C0008616C6C2070617261F0
:1072B000206973206F6B00002DE9F04107460D46F1
:1072C000164606B15DB9EE212AA0FBF795F810B17C
:1072D0002EA000F08DFE4FF0FF30BDE8F081384663
:1072E000FFF7E8FE80462A4641463046F9F70DFA98
:1072F00050B9F4211FA0FBF77FF818B1394627A039
:1073000000F090FE0020E8E73846FFF70DFE044647
:10731000B4F1FF3F0AD1FB2116A0FBF76DF810B1C5
:1073200026A000F065FE6FF00100D6E7264A02EBCA
:10733000C4025178244A02EBC4025068F9F740FBBA
:10734000214A02EBC40250782946884201DA0246FB
:1073500000E00A4690461C4901EBC40142464868D9
:107360003146F9F774FA1821184800F0AFF80020F8
:10737000B3E700002E2E5C4D4F445C5372635C6D8E
:107380006F645F7379732E63000000007061726137
:107390006D65746572206572726F720070617261E2
:1073A0005F69645B25645D2C70617261206E6F742F
:1073B000206368616E67656400000000706172613F
:1073C0002045727200000000E09C0008184D00206B
:1073D0000EB540F20F111BA0FBF70EF828B11F48A5
:1073E000428801881EA000F01DFE4FF4887115A090
:1073F000FBF702F878B11948407A1849097A174A18
:10740000D279CDE90021029014488379427901793B
:107410001BA000F007FE40F213110AA0FAF7ECFFE0
:1074200020B10E490A3121A000F0FCFD4FF48A7111
:1074300004A0FAF7E1FF20B1084841691EA000F05E
:10744000F1FD0EBD2E2E5C4D4F445C5372635C6D9E
:107450006F645F7379732E6300000000184D002085
:10746000706172615F6372633A307825782C2070A6
:107470006172615F73697A653A307825780000003F
:10748000626C655F6D61633A307825783078257875
:1074900030782578307825783078257830782578D8
:1074A000307825783078257800000000626C655FC0
:1074B0006E616D653A257300626C655F6164765F2D
:1074C000496E74657276616C3A2564002DE9F0416D
:1074D00004460D464FF0000814B90120BDE8F081C4
:1074E0006580A91EA01C00F069FD8046A4F80080FC
:1074F0001248FFF739FD10B11048FFF77BFDAAB223
:1075000021460E48FFF7AAFD06460EB947F00107CF
:107510000B48FFF729FD10B10948FFF76BFDAAB230
:1075200021460748FFF79AFD06460EB947F00207C5
:10753000032F01D00220D1E70020CFE700F4030899
:1075400000F0030800BFFEE77047704708B5084920
:107550000968C9084FF47A72B1FBF2F14143009116
:1075600000BF00BF00994A1E00920029F9D108BD52
:107570000800002000B585B000BF1048806940F0C9
:1075800004000E4988610846806900F004000090FC
:1075900000BF00BF04200190012002900020039052
:1075A0000220049001A90648FCF76CFC012204218A
:1075B0000348FCF716FE05B000BD000000100240B5
:1075C0000008014000B585B000BF1048806940F058
:1075D00004000E4988610846806900F004000090AC
:1075E00000BF00BF012001900948029000200390D5
:1075F00001A90848FCF746FC022211460620FCF7C8
:10760000E4FE0620FCF7D1FE05B000BD00100240EC
:10761000000011100008014010B511481149086020
:107620004FF48270486000210E488160C1600221E1
:10763000016101214161490281613821C16100215B
:107640000162416281620A21C162FDF7C4FB054803
:107650000068006840F0400002490968086010BDF9
:1076600000300140444C002070B505460C464FF4F4
:107670007A73224629460448FDF72CFC10B14FF0DE
:10768000FF3070BD2046FCE7444C002010490968DB
:10769000096821F040010E4A126811600C4909681E
:1076A00009684FF6C7721140094A1268116008490B
:1076B000096809680143064A1268116004490968AB
:1076C000096841F04001024A1268116070470000E9
:1076D000444C002070B505460C464FF47A732246A0
:1076E00029460448FDF71BFD10B14FF0FF3070BD77
:1076F0002046FCE7444C0020F8B504460E461546EB
:107700006068B0F5827F0DD1A068B0F5004F03D05E
:10771000A068B0F5806F05D12068006820F04000B7
:10772000216808606068B0F5827F11D1A068B0F56B
:10773000806F0DD13346002201212046009500F0D4
:107740002EF898B1606D40F0200060650320F8BD10
:107750003346002280212046009500F020F828B111
:10776000606D40F0200060650320F0E70020EEE748
:10777000F8B504460D4616462B46002280212046C9
:10778000009600F00CF828B1606D40F020006065B4
:107790000320F8BD0020FCE70146012070472DE9D9
:1077A000F04104460E4617461D46DDF818803EE0BF
:1077B000681CD8B3FCF71CFDA0EB0800A84200D25F
:1077C000A5BB2068406820F0E00021684860606840
:1077D000B0F5827F0DD1A068B0F5004F03D0A0684E
:1077E000B0F5806F05D12068006820F04000216866
:1077F0000860A06AB0F5005F0DD100BF2068006886
:1078000020F40050216808602068006840F40050AF
:107810002168086000BF012084F8510000BF0020EB
:1078200084F8500000BF0320BDE8F081FFE7206826
:1078300080683040B04201D1012000E00020B84211
:10784000B6D10020F0E770477CB506460D46B5F589
:10785000407F02DD4FF4407000E02846054640F2CC
:1078600001610C48F9F7ACF800240BE0325D0AA185
:107870006846F8F77BFD074800EB4400BDF80010B0
:107880000180641CAC42F1DB0020024981F8000653
:1078900008467CBD505300202530325800000000BF
:1078A0002DE9F04780460E46402E0ADD442139A0DE
:1078B000FAF7A2FD10B140A000F09AFB0020BDE84D
:1078C000F08740214448F9F77BF8304606EBD07149
:1078D0004910A6EB410149B14C212EA0FAF78CFDCD
:1078E00010B13EA000F084FB0020E8E70027B94675
:1078F0004BE018F80740412C05DB462C03DCA4F1D3
:107900003700C4B216E0302C05DB392C03DCA4F1BF
:107910003000C4B20EE00D2C01D00A2C01D100249D
:1079200008E061211BA0FAF767FD18B1214633A0DA
:1079300000F05EFB7F1C18F80750412D05DB462D3B
:1079400003DCA5F13700C5B216E0302D05DB392D7B
:1079500003DCA5F13000C5B20EE00D2D01D00A2DDB
:1079600001D1002508E074210AA0FAF745FD18B1FD
:1079700021462BA000F03CFB45EA0410C2B2484669
:1079800009F1010914490A547F1CB742B1DB1248BE
:1079900095E700002E2E5C4D6964646C655C73791C
:1079A000735F636F6D6D6F6E5C7379735F636F6D23
:1079B0006D6F6E2E6300000053747232486578203C
:1079C0006C656E67746820697320746F6F206C61DA
:1079D00072676520212121005159002053747232B1
:1079E000486578206C656E677468206973206E6FD7
:1079F00074207269676874202121210053747232E7
:107A000048657820646174615B25645D206E6F74E5
:107A10002072696768742031202121210000000054
:107A20005374723248657820646174615B25645DCB
:107A3000206E6F74207269676874203220212121C2
:107A40000000000070B505460C462046F8F789FE98
:107A50000646324621462846F8F7FBFF70BD70B552
:107A600004460D4629462046F8F73DFE70BD30B568
:107A70008FB00546002401200590000406900020E8
:107A8000079002200C90C1030D910E9505A8FCF7FC
:107A900055FF04460CB100BFFEE70F200090022006
:107AA0000190002002904FF4806003900020049029
:107AB00002216846FCF70CFE04460CB100BFFEE74D
:107AC0000FB030BD10B5FCF7C9FB10BD08B10149BE
:107AD000086070474426002001480249086070474A
:107AE0000400FA050CED00E01148006840F00100C8
:107AF0000F490860084640680E4908400C49486034
:107B0000084600680C4908400949086008460068B2
:107B100020F4802008600846406820F4FE00486099
:107B20004FF41F008860C8030449086070470000D4
:107B3000001002400000FFF8FFFFF6FE08ED00E035
:107B400010B50248FDF75EFE10BD0000044C002099
:107B500010B50268204B98420ED0204B98420BD0B3
:107B6000B0F1804F08D01E4B984205D01D4B984273
:107B700002D01D4B984203D122F070024B681A4389
:107B8000154B98420ED0154B98420BD0B0F1804F58
:107B900008D0134B984205D0124B984202D0124B9A
:107BA000984203D122F44072CB681A4322F080033A
:107BB0004C6943EA040202608B68C3620B6883620B
:107BC000054B984202D0054B984201D10B690363E3
:107BD0000123436110BD0000002C0140003401402E
:107BE0000004004000080040000C004070B505464D
:107BF0006C6A0020E085E0842046FDF757FF70BDE9
:107C00000168C96821F490710268D160016849690E
:107C100021F0010102685161202180F83A1070477B
:107C200010B504462068C06820F040002168C86094
:107C3000202084F839002046FEF76DF9002010BDA1
:107C400070B5044694F83A0022284AD1A068B0F5ED
:107C5000805F13D1A56A206940B920684068C0F3ED
:107C600008002880A06A801CA06219E02068406893
:107C7000C0B22880A06A401CA06211E0206938B917
:107C800020684068C1B2A26A501CA062117007E06F
:107C90002068406800F07F01A26A501CA062117049
:107CA000E08D401E80B2E085C8B92068C06820F031
:107CB00020002168C8602068C06820F480702168B6
:107CC000C8602068406920F00100216848612020D8
:107CD00084F83A002046FEF761F8002070BD0020CD
:107CE000FCE70220FAE7000070B504462168096944
:107CF00021F44051E2681143226811612269A168B0
:107D00001143626941EA02052168C96841F20C62C7
:107D1000914329432268D1602168496921F4407167
:107D2000A269114322685161564A2168914254D197
:107D3000FCF7AAFD00EBC00101EB001162689200A4
:107D4000B1FBF2F100EBC00202EB001263689B0092
:107D5000B2FBF3F26423B2FBF3F202EBC20303EBD8
:107D60000212A1EB8201322202EB01116422B1FB6B
:107D7000F2F101F0F00100EBC00202EB00126368C7
:107D80009B00B2FBF3F26423B2FBF3F201EB0212AD
:107D900000EBC00101EB001163689B00B1FBF3F144
:107DA00000EBC00303EB00136668B600B3FBF6F309
:107DB0006426B3FBF6F303EBC30606EB0313A1EB58
:107DC0008301322303EB01116423B1FBF3F101F0D2
:107DD0000F0111442268916053E0FCF745FD00EB70
:107DE000C00101EB001162689200B1FBF2F100EBFF
:107DF000C00202EB001263689B00B2FBF3F2642343
:107E0000B2FBF3F202EBC20303EB0212A1EB82011D
:107E1000322202EB01116422B1FBF2F101F0F00118
:107E200000EBC00202EB001263689B00B2FBF3F2AE
:107E30006423B2FBF3F201EB021200EBC00101EB91
:107E4000001163689B00B1FBF3F100EBC00303EB8F
:107E500000136668B600B3FBF6F36426B3FBF6F3D3
:107E600003EBC30606EB0313A1EB8301322303EB01
:107E700001116423B1FBF3F101F00F0111442268F9
:107E8000916070BD00380140014691F83900212809
:107E90002CD18868B0F5805F0FD10A6A1088C0F3D2
:107EA00008000B685860086918B9086A801C0862E5
:107EB00009E0086A401C086205E00B6A581C086269
:107EC00018780B685860C88C401E80B2C88458B9B6
:107ED0000868C06820F080000B68D8600868C06837
:107EE00040F040000B68D860002070470220FCE79B
:107EF0002DE9F04104460D4617469846069E21E0BE
:107F0000701CF8B12EB1FCF773F9A0EB0800B04279
:107F100018D92068C06820F4D0702168C860206833
:107F2000406920F0010021684861202084F8390070
:107F300084F83A0000BF002084F8380000BF032016
:107F4000BDE8F081206800682840A84201D10120E6
:107F500000E00020B842D3D00020F1E710B50024A3
:107F60000C48FDF7AFFD00BF01E0641C00BF0948ED
:107F7000FDF79DFD2028F8D100BF002401E0641C1E
:107F800000BF012204490348FDF7D0FE0028F6D1C6
:107F900000BF10BD684B00202200002010B5024831
:107FA000FBF739F910BD0000A84B002010B50248BE
:107FB000FBF731F910BD0000A84B002010B50246B8
:107FC0000B464FF6FF7109E010784840C0B2064CEE
:107FD00034F8100080EA21215B1E521C002BF3DCD8
:107FE000C84380B210BD00004C26002000BFFEE751
:107FF0000FB408B50948007802280BDB0848007860
:1080000040B103A800900220009A0299FAF736FACC
:108010000020009001B05DF814FB0000392600201C
:10802000382600200FB408B50948007804280BDB77
:108030000848007840B103A800900420009A0299F3
:10804000FAF71CFA0020009001B05DF814FB000064
:108050003926002038260020490050EAC12018BFE8
:1080600004204A0D18BF40F0010040F2FF72B2EB4D
:10807000515F08BF40F00200012808BF052070478B
:1080800002480068C0F30220704700000CED00E0D9
:1080900010B5002804DB0A07130E054A135406E046
:1080A0000A07140E034A00F00F031B1FD45410BD1F
:1080B00000E400E018ED00E070B586B0044600254D
:1080C0000020019002900120039004940590FBF79A
:1080D00055FE002607E001A902A8FBF795FD05461D
:1080E00005B902E0761C032EF5DB00BFFBF7E4FDCB
:1080F00015B1012006B070BD0020FBE770B5054644
:108100000C460026FBF73AFE2246002329460220B1
:10811000FBF7DCFD0646FBF7CFFD0EB1032070BD7B
:108120000020FCE730380A2801D2012070470020E7
:10813000704700BF7047000010B504468E2104A0B0
:10814000FAF75AF918B1214603A0FFF751FF10BD05
:108150006D61696E2E63000063616E5F6572726FA0
:10816000723A3078257800002DE9F04389B007464F
:108170000E4690461C460025B6F5987F02D109B000
:10818000BDE8F0838DF80470681CC5B2CDF80560B9
:10819000281DC5B28DF80940681CC5B2224641466B
:1081A0000DF10A00F8F753FB2819C5B27E210BA088
:1081B000FAF722F958B121464046FFF745FB8146C0
:1081C000234632463946009006A0FFF72BFF29468A
:1081D00001A8FEF7F1FA00BFD1E700006D61696EFA
:1081E0002E63000072782063616E5F69645F74794A
:1081F00070653A25642C63616E5F69643A30782556
:10820000782C646174615F6C656E3A25642C6461DE
:1082100074613A2573000000704770477047000092
:1082200010B504460420FDF7DEF90148046010BDD6
:108230001800002030B50446002504E04FF47A70A1
:1082400000F004F86D1CA542F8D330BD70B50346AC
:1082500000224FF0E02675690D4E366803FB06F4E8
:108260004FF0E026B16910E04FF0E026B069884297
:108270000BD0884202D20E1A324402E02E1A0E446B
:1082800032440146A24200D300E0EDE700BF70BDDA
:10829000180000207047000000BF054A126802F075
:1082A0004002002AF9D0C2B2014B1B1D1A60704770
:1082B000003801400148006870470000482600204F
:1082C00010B5FDF747FA10BD704770B504460D466E
:1082D0006068F0B1E26861682846F8F7FDFA606806
:1082E000E1680844E2682168236902FB03118842BF
:1082F00001D1206802E06068E1680844606060685D
:10830000A168884201D1002000E060686060002020
:1083100070BD0A20FCE770B504460D466068A16890
:1083200088421CD0E268A0682946F8F7D5FA606850
:1083300008B9A06800E060686060A068E16808446F
:10834000E2682168236902FB0311884201D1206899
:1083500002E0A068E1680844A060002070BD092028
:10836000FCE72DE9F04104460E4617461D4664B170
:1083700007FB06F12846F8F723FBE760266100209B
:108380006060A5602560BDE8F081FF20FBE770B567
:1083900004460D46294604F5CB60FFF7BCFF08B93B
:1083A000002070BD0820FCE710B504460CB917206A
:1083B00010BD6078042804D06078082801D014200B
:1083C000F6E74FF4C860005918B140F23C6000591C
:1083D00008B91620ECE7D4F8200610B91A48C4F8FA
:1083E000200640F22460005918B9184940F2246070
:1083F00001514FF4C560005918B915494FF4C560D3
:10840000015140F22C60005918B9124940F22C6019
:1084100001514FF43071201DF8F7F4FA4FF4307128
:1084200004F53170F8F7EEFA9A2104F28450F8F767
:10843000C7FA04F26C631422202104F5CB60FFF725
:1084400090FF0020B4E70000C98200089582000870
:108450001D8200081B82000830B585B005462846FD
:1084600001F03BF8044604E06946284600F00FF8A6
:108470000443694605F5CB60FFF727FF0A28F3D1CF
:10848000284600F047F80443204605B030BD38B513
:1084900004460D46287A207100BF00BF00BF00BF10
:1084A00005F10C000090AB7A2078A11D2A6800F03D
:1084B00019FD40BB00BF00BF207D30B101280BD0AB
:1084C000022810D003281CD114E000BF00BF2946A9
:1084D000204600F0EBFF38BD00BF00BF2946204614
:1084E00000F099FFF7E700BF00BF2946204600F0E3
:1084F000C9FEF0E700BF00BF2946204600F02AFF72
:10850000E9E700BF00BF4FF4C76001592920884741
:108510002920E0E72DE9FC47044694F86503042888
:1085200006D094F86503052802D01020BDE8FC872A
:1085300000BF00BF092625782078602800D1452596
:108540004FF0FF08204600F0E9FA84F8D4022046F4
:1085500000F0E4FA804600BF00BF00BF00BFB8F1E2
:10856000000F06D0B8F1010F3CD0B8F1020F76D160
:1085700090E0B4F86613A4F8D612B4F86613A4F821
:10858000C81200BF00BF207804F55E7301AA04F290
:10859000C62100F0CEFB00B136E1B4F8C8220021BC
:1085A000284600F08AFA014694F8C802084400F010
:1085B000FF0A94F8C412504600F056FA074604F534
:1085C0003670009094F8C42260784FF4C86151F876
:1085D00004C03B460199E04708B9002000E00920AB
:1085E000064611E100BF00BFB4F86613A4F8D61226
:1085F000002184F8611394F8C402012806D105F023
:10860000010008B9062107E0052105E005F0010099
:1086100008B93E2100E03D21A4F8C812B4F8C81200
:10862000A4F8681300BF00BF207804F55E7301AAA8
:1086300004F2C62100F07DFB00B1E5E0012184F8E1
:108640006013102184F8651300BF00BF04F5367075
:10865000009094F8C412012902D1082101E0CFE072
:1086600040210B4694F8C42260784FF4C8610F593A
:108670000199B84708B9002000E00920064640F2F9
:108680003C6108598047C4F86C030EB900204DE7DF
:1086900009204BE740F23C6108598047014694F8B5
:1086A0004426D4F874031044814201D200203DE7EF
:1086B00094F8600300F00F0184F8D21294F860037C
:1086C000FF2801D1002002E094F86003401C84F8E8
:1086D000600300BF00BF94F8C40201281ED105F05A
:1086E000010109B9072100E00621084600BF00BFCB
:1086F000B4F86623B4F86813511AA4F8C81200BF7E
:1087000000BFB4F8C812814201DB024601E0B4F8B0
:10871000C822A4F8C82200BF00BF18E005F001017C
:1087200009B93F2100E03E210846B4F86623B4F8B9
:108730006813511AA4F8C812B4F8C812814201DBB8
:10874000024601E0B4F8C822A4F8C82200BF00BF66
:1087500000BF00BF00BFB4F8682304F55E71531872
:10876000207801AAB23900F0E4FA00B14CE0B4F884
:108770006813B4F8C8020844A4F8680394F8D21245
:1087800040F24560005D81420AD1102184F86513F2
:1087900000BF00BF40F23C6108598047C4F86C0339
:1087A00005F0010008B9012000E00220814694F89C
:1087B000C41294F8C8224A44D0B200F055F9824657
:1087C00004F53670009094F8C42260784FF4C861C4
:1087D0000F5953460199B84708B9002000E0092015
:1087E000064640F23C6108598047C4F87403B4F867
:1087F0006813B4F86603814200DB05E0002095E6CB
:1088000000BF00BF092091E6002184F8651300BF76
:1088100000BF84F8601384F861134FF4C5600096BC
:108820000259002304F53171032000F0D1FF3046D6
:108830007CE670B504460D4694F8650318B100BF98
:1088400000BF112070BDE889B0F5017F01DD08206F
:10885000F8E7287884F8C402E989A4F86613EA895D
:1088600005F1100104F55E70F8F736F80522691C71
:1088700004F2CA20F8F730F8042184F8651300BF29
:1088800000BF0020DEE710B50020FBF77FFD10BD24
:1088900098B01C2111A8F8F7B5F8FBF7EBFC4FF4E2
:1088A000E010FFF7E4F84820FFF7BAFC4FF4E1309E
:1088B00001F05AF84FF4FA610420FDF757FBFDF779
:1088C0004BFB4D4800F08AFE4C4800F087FE4C48B8
:1088D00000F084FEFAF7D2F94A48FDF71DFB4A483A
:1088E000FFF7F4F8FAF7F0F90120FAF713FAFBF7BB
:1088F00005FD0020FBF73CFD41F61F410920FDF777
:108900005BF84248FEF7E4F94148FCF7C5FE414AEE
:1089100041494248FAF75CFFFDF738FFFAF78AFF52
:1089200004464CB1BE213EA0F9F766FD10B13EA051
:10893000FFF75EFB00BFFEE7FAF7DCFF04464CB131
:10894000C42137A0F9F758FD10B13BA0FFF750FB49
:1089500000BFFEE7FEF7DAFBC8213B48FDF742F80F
:1089600041F288313948FDF73DF8CD212CA0F9F7C7
:1089700043FD30B1FFF79EFC0546294634A0FFF7C2
:1089800051FB37E0FDF7F2FE00BF1D4800F0D9FDB6
:1089900058B901A91A4800F02BFE0546002D03DD49
:1089A000E9B201A8FCF7AAFE00BF00BF00BF134850
:1089B00000F0C7FD58B901A9104800F019FE05469E
:1089C000002D03DDE9B201A8FEF710F800BF00BFDB
:1089D00000BF094800F0B5FD58B901A9064800F0EC
:1089E00007FE0546002D03DDA9B201A8FDF7D0FA68
:1089F00000BF00BFC6E700004C280020D830002090
:108A000064390020A1990008255F000851990008E9
:108A10002999000839810008198200086981000835
:108A20006D61696E2E63000063616E5F696E6974CB
:108A30005F6572726F72000063616E5F7374617262
:108A4000745F6572726F7200878800082D9200084B
:108A5000696E69742066696E69736865642C207636
:108A600065723A307825780002460020012906D147
:108A7000082A01D8134600E0082318461CE0082AFB
:108A800001DC104618E00C2A01DC0C2014E0102A4E
:108A900001DC102010E0142A01DC14200CE0182A5C
:108AA00001DC182008E0202A01DC202004E0302A24
:108AB00001DC302000E04020704730B503461C4602
:108AC000602B00D1452404F0010031B1012910D000
:108AD000022919D003291DD119E0451CE8B2C0F1C3
:108AE0000805954201DA012500E000250544E8B2B9
:108AF00012E0851CE8B2B2F5805F01DB042500E0DE
:108B000000250544E8B207E0451CE8B204E0C51CB6
:108B1000E8B201E0002000BF00BF30BD01460220E6
:108B20000A780B78602B00D1452291F8603323BB83
:108B300002F00103ABB191F8C432012B08D1B1F8B6
:108B40006633062B01DD012300E0002318461DE0FB
:108B5000B1F866333D2B01DD012300E00023184608
:108B600014E091F8C432012B08D1B1F86633072B19
:108B700001DD012300E00023184607E0B1F8663369
:108B80003E2B01DD012300E0002318467047F0B5BD
:108B9000034609251C46002968D0002A66D0602BB0
:108BA00000D1452400BF00BF04F001008E7B36B128
:108BB000012E2ED0022E22D0032E53D13CE00E8A5D
:108BC000C0F10707BFB2BE4208DC8F7B0E7C67F3A3
:108BD0001F16F7B201F1120637540EE08E7B002704
:108BE00007EB0616F7B201F11206375491F810C0E0
:108BF000461C01F1120707F806C0002534E00F7B80
:108C00008E7B47EA0616F7B201F1120637540025AB
:108C10002AE00E8AC6F303278E7B47EA0616F7B2D0
:108C200001F11206375491F810C0461C01F11207E9
:108C300007F806C0002517E08F7A8E7B47EA0616F4
:108C4000F7B201F11206375491F80BC0461C01F13E
:108C5000120707F806C091F80DC0861C07F806C079
:108C6000002501E0092500BF00BF00BF2846F0BD78
:108C7000F0B5044609262546602D00D1452500297A
:108C800055D0002B53D005F001001F5C4FEA171C94
:108C900081F80EC000BF00BF8F7B37B1012F11D00C
:108CA000022F34D0032F3ED11DE0082A03DC1F5CC5
:108CB00007F00F0701E0471CDF5D0F82002600BFB1
:108CC00000BF32E0471CDF5D13F800C00CF00F0C52
:108CD00047EA0C2CA1F810C0871CD71B4F80002638
:108CE00000BF00BF21E01F5C07F00F078F72471C19
:108CF00013F807C081F80BC0871C13F807C081F870
:108D00000DC0D71B4F80002600BF00BF0DE01F5CC9
:108D100007F00F0C81F80CC0471CD71B4F800026B2
:108D200000BF00BF01E0092600BF00BF00BF304602
:108D3000F0BD2DE9F04107460C4615461E4606B12A
:108D400015B90920BDE8F08100BF00BF452F0CD048
:108D500006DC142F0CD0282F2FD0352F5CD13DE00E
:108D6000592F17D0602F57D14CE0A079A07400BFC5
:108D70002079802141EA0021A07941EAC00061798F
:108D80000843217A012901D1402100E00021084354
:108D9000286043E020798106207A012801D1CE2085
:108DA00000E0CD2041EA0041A07941EA002061794C
:108DB00008432860E079A07430E020798106207AA9
:108DC000012801D1DA2000E0DB2041EA0041A0794E
:108DD00041EA00206179084328601FE02079802162
:108DE00041EA0021A07941EAC00061790843217A73
:108DF000012901D1402100E0002108432860E079E9
:108E0000A0740BE06079217900EB01202860A07943
:108E1000A07400BF00BF01E0092093E700BF324605
:108E200021463846FFF7B3FE32462146384600F069
:108E300001F887E72DE9F04705460C461646092755
:108E4000A846002E4BD0602D01D14FF04508A07BE5
:108E500030B1012813D0022820D003283CD12CE0C7
:108E6000628800214046FFF728FE04F1120100EB62
:108E70000109628831464846F7F72EFD2DE06288E9
:108E800001214046FFF719FE04F1120100EB010930
:108E9000628831464846F7F71FFD1EE062880221CE
:108EA0004046FFF70AFE04F1120100EB0109628857
:108EB00031464846F7F710FD0FE06288032140462F
:108EC000FFF7FBFD04F1120100EB01096288314656
:108ED0004846F7F701FD00E000BF00BF0027384615
:108EE000BDE8F0872DE9F04707460C461546984641
:108EF000089E04B116B90920BDE8F08700BF00BF85
:108F0000B946B9F1450F45D009DCB9F1140F10D0BD
:108F1000B9F1280F2FD0B9F1350F60D106E0B9F1C2
:108F2000590F17D0B9F1600F59D146E03178E1718E
:108F300000BFC5F302202071C5F3C201A17105F085
:108F400007016171C5F3801008B1012100E0022121
:108F5000217246E03178E171C5F382602071C5F37A
:108F60000740CE2801D1012100E002212172290A07
:108F7000A171657135E0C5F382602071C5F30740CA
:108F8000DA2801D1012100E002212172290AA17110
:108F9000657126E0C5F302202071C5F3C201A171FD
:108FA00005F007016171C5F3801008B1012100E0EF
:108FB000022121723178E17113E0C5F302202071A2
:108FC000A571290A6171C5F3801008B1012100E083
:108FD000022121723178E17100BF00BF01E006205B
:108FE0008AE700BF3346424621463846FFF740FE37
:108FF00032462146384600F004F800BF00BF00208A
:109000007AE72DE9F04706460C4615464FF0090869
:109010003746602E00D14527002C56D0002D54D065
:10902000A07B30B1012816D0022826D0032848D1D1
:1090300035E000BF00BF228A00213846FFF73DFD22
:1090400000EB0509228A494604F19200F7F744FC37
:109050004FF0000838E000BF00BF628801213846A9
:10906000FFF72BFD00EB05096288494604F1120069
:10907000F7F732FC4FF0000826E000BF00BF62881F
:1090800002213846FFF719FD00EB050962884946C1
:1090900004F11200F7F720FC4FF0000814E000BFC5
:1090A00000BF628803213846FFF707FD00EB050982
:1090B0006288494604F11200F7F70EFC4FF00008F1
:1090C00002E04FF0090800BF00BF4046BDE8F0874E
:1090D00010B50446242104A0F9F78EF918B12146F1
:1090E00009A0FEF785FF10BD2E2E5C4D4F445C534A
:1090F00072635C6D6F645F63616E646174617072F2
:109100006F636573732E63003135373635207061B8
:10911000727365206572723A253034780000000061
:1091200070B504463D211BA0F9F766F910B121A0E6
:10913000FEF778FFA07B00281DD1402115A0F9F78C
:109140005BF940B1E578A07845EA0022238AA17B4B
:109150001CA0FEF767FF002506E004F11300415D47
:1091600026A0F7F7F7F86D1C208AA842F5DC25A0A9
:10917000F7F7F0F80CE04D2106A0F9F73DF938B10A
:10918000E378A07843EA0022A17B1FA0FEF74AFF04
:1091900070BD00002E2E5C4D4F445C5372635C6DBD
:1091A0006F645F63616E6461746170726F63657335
:1091B000732E630070617273652066696E697368EF
:1091C00000000000706172736520737563636573DE
:1091D000732E72736C743A307825782C6672616DD8
:1091E000655F69643A307825782C6D73675F737AB0
:1091F0003A307825782C646174613A002530325811
:10920000000000000D0A0000706172736520666145
:10921000696C2E72736C743A307825782C667261A2
:109220006D655F69643A30782578000010B50C48A8
:109230000068401D0A49086038210AA0F9F7DCF8E7
:1092400020B10748016809A0FEF7ECFE0448006859
:109250000B49884202D100200149086010BD00007E
:10926000040000206D61696E2E6300006D6375203F
:1092700072756E207365636F6E64733A2564730054
:10928000803A0900F8B504460E46002594F8A5007A
:1092900000F0020008B9222550E094F8A000401C1C
:1092A0000F2801DD002002E094F8A000401C84F8A3
:1092B000A00000BF00BF00BF00BF94F8A00000F0F6
:1092C0000F01A07C814201D0262537E02289B4F825
:1092D000A83004F1B8015818A039F7F7FDFAB4F82E
:1092E000A81020890844A4F8A800B4F8A810B4F87D
:1092F000A600814213DB00200090B4F8A630211DA7
:109300000120D4F8202600F063FA4FF43071201DBC
:10931000F7F778FB0021C4F8B0100020F8BD00BFBB
:1093200000BF40F24560005D00B100BF40F23C610B
:1093300008598047C4F8B0002846EFE74FF4C760EB
:10934000015928468847002184F8A51000BF00BFB6
:109350002846E3E72DE9F04104460F46062600BF04
:1093600000BF00BF00BF207C78B3012802D00228D4
:109370003BD128E094F86103401C84F86103254642
:1093800095F8611340F24660405D814201DA0020A9
:109390000CE04FF4C76041590720884700231A4664
:1093A000194605F5317000F00BFA0720072802D0A6
:1093B0000020BDE8F08140F23C6108598047C4F8C4
:1093C0006C03072613E0082611E0FFE7617C84F8B0
:1093D0006413E17C84F8631305230022012104F562
:1093E000317000F0EDF90020E3E7312600BF00BF47
:1093F00000231A46194604F5317000F0E1F94FF4E4
:10940000C760015930468847002184F8A51000BF85
:1094100000BF3046CDE738B504460D46B4F8A60087
:10942000B0F5017F06DD4FF4C76001593020884751
:10943000302038BD94F8A50000F0020080B100BFD4
:1094400000BF4FF4C76001590620884706200090EE
:10945000B4F8A630211D0120D4F8202600F0B8F978
:10946000228904F1180104F1B800F7F735FAE18A0E
:10947000A4F8A6102189A4F8A81000BF00BF0021FD
:1094800084F8A01084F8A11000200090B4F8A63051
:1094900040F224600259211D022000F099F900BF1A
:1094A00000BF204600F0D5F80020C2E738B50446DA
:1094B0000D4600BF00BFE28A04F1980104F52F7049
:1094C000F7F70AFA00200090E38A211D0520D4F85E
:1094D000202600F07DF9002038BD38B5044694F808
:1094E0006503102812D1D4F86C0378B14FF4C96029
:1094F000005B58B140F23C61085980474FF4C961A4
:10950000095BD4F86C231144884201D8002038BD8F
:1095100000BF00BF00BF00BF002184F8601302201D
:109520000090B4F8663304F531710120D4F8202698
:1095300000F04EF94FF4C76001590220884702201D
:10954000E5E70146D1F8880808B9012070470020F6
:10955000FCE70146D1F88808202801D10120704796
:109560000020FCE770B504460E4615462046FFF77E
:10957000F0FF00B170BD402D01DD402000E0284625
:10958000054604F684042068401C20602068C1174A
:1095900000EBD1614911A0EB411121606068401CD2
:1095A00060602168A4F6840401EB011104EB8100E2
:1095B0004421F7F727FAD4F8841801EB011104EBE2
:1095C0008101081D2A463146F7F741F9D4F884088D
:1095D00000EB001044F8205000BFCBE74FF0FF3104
:1095E000C0F88018C0F884180021C0F888187047A7
:1095F00070B504460D462046FFF7A3FF08B10020D2
:1096000070BD04F508642068401C20602068C11704
:1096100000EBD1614911A0EB41112160A068401E0F
:10962000A0602068A4F5086400EB001054F8202026
:10963000D4F8800800EB001004EB8000011D2846E0
:10964000F7F705F9D4F8800800EB001054F8200073
:10965000D6E77CB5044694F8650340F0040184F82D
:10966000651300BF00BF032184F8921540F24560E6
:10967000015D84F88F1594F8441684F89115617B88
:1096800084F88B15217B84F88915E17A84F88A1592
:10969000A17A4FF4B1600155A17B84F88C1540F29A
:1096A0004560015D84F8A41000BF00BF207804F578
:1096B0005E7301AA04F28451FFF73BFB48B194F8B2
:1096C000650320F0040184F8651300BF00BF092082
:1096D0007CBD00BF00BF40F286510A5B20780321A9
:1096E000FFF7EBF9064604F2965000902279607875
:1096F0004FF4C8610D5933460199A84794F86503A2
:1097000020F0040184F8651300BF00BF0020DFE7EC
:109710002DE9FE4F05460E461F46DDF830804FF01E
:109720000009CA4600240020019002908346A94601
:10973000B246082F01DD082000E03846044600202C
:10974000019002902246414601A8F7F780F83521A2
:109750000CA0F8F751FE48B1214601A8FEF774F8B5
:109760000246214600900FA0FEF75CFC234601AAAA
:1097700051464846FAF7DEF800F0FF0B0020BDE83E
:10978000FE8F00002E2E5C4D4F445C5372635C6D67
:109790006F645F63616E6461746170726F6365733F
:1097A000732E630073656E642063616E2064617460
:1097B000613A25642C646174613A257300000000ED
:1097C00000F89C1F427043719C3800BF00BF704777
:1097D0002DE9F04180460C4615461E46069F00BF07
:1097E00000BF002D6FD0B8F1010F09D0B8F1020F02
:1097F0004AD0B8F1030F68D0B8F1050F7CD123E04F
:1098000040488773068220783E4908700220887499
:109810000522A11D3B48401CF7F75EF8082204F121
:109820000C013848801DF7F757F8324604F1B401AF
:1098300034481330F7F750F8002084F8A10000BF37
:1098400000BF3048A84759E02F4887730682207828
:109850002D490870002088740522A11D2A48401C4B
:10986000F7F73AF8082204F10C012748801DF7F7B2
:1098700033F8324604F52E712448F7F72DF800BF6F
:1098800000BF2148A84739E02078214908700846E0
:10989000C681012008740522A11D1D48401CF7F750
:1098A0001BF8082204F10C011948801DF7F714F881
:1098B00094F8A10040F0020084F8A10000BF00BFAE
:1098C0001348A8471AE01AE0FFE7124887730320FD
:1098D0001049C8730522A11D0E48F6F7FDFF0822A6
:1098E00004F10C010B48801DF6F7F6FF00BF00BF26
:1098F0000848A84702E0FFE7BDE8F08100BF00BFCD
:10990000FAE70000945B0020B45D0020CB5F0020EC
:10991000D45F0020E65F002010B501460A784B783E
:109920000B704A7010BD000010B590B00446402185
:109930006846F7F767F840216846FBF7BBFE402210
:1099400069460248FFF70EFE10B010BDD830002067
:1099500070B504460D462A4621460248FFF702FE2E
:1099600070BD00006439002010B5044609480A495A
:1099700008600846446000218160C1600161816126
:109980000C214161FCF744F9012204490248FCF72B
:10999000CDF910BD00380140684B002022000020A6
:1099A00070B504460D462A4621460248FFF7DAFD07
:1099B00070BD00004C28002010B50248FAF746FCA4
:1099C00010BD0000CC4C002010B500290AD008784A
:1099D000002807D005487844F7F7E0FF002801D0B9
:1099E000002010BD0248784410BD00008E04000025
:1099F0008604000010B500290AD00878002807D096
:109A000005487844F7F7CAFF002801D0002010BDB0
:109A10000248784410BD0000720500006A0500008D
:109A20004FEA41034FEA5353A3F58063D3F11E037A
:109A3000C8BFD3F1210C0CDD4FF0004242EAC12235
:109A400042EA505232FA03FC8CEAE17CACEBE17062
:109A50007047102BC4BF0020704703F5787CBCF121
:109A6000FF3F04D06FF0004282EA2100704770B5DA
:109A700000F0C6F84992248000207047F2E710F009
:109A8000004248BF4042B0FA80F310FA03F10AD016
:109A9000C3F11D0303F580634FEA415002EB03520B
:109AA00002EBD12170474FF000007047DFF848C14A
:109AB00070B51CEA111E1EBF1CEA13159EEA0C0F9E
:109AC00095EA0C0F00F06F8081EA030423EA4C133F
:109AD0004EEAD47E21EA4C1141F4801143F4801304
:109AE000AE44A1FB024CA0FB0365AEF17F7E3619AC
:109AF00055EB0C05A1FB034C4CF10003A0FB021C31
:109B000016EB0C06654153F10003094218BF46F0FD
:109B1000010613F4007F0BD14FEA03314FEA053001
:109B2000340341EA155140EA16506FF003020AE08F
:109B30004FEAC3214FEAC520F40241EA555140EAF9
:109B400056506FF0020202EB2E4201EB025585EAFD
:109B5000CE710AD05FEA440C18BF24F0004450F1E3
:109B6000000041F1000120EAD47040F2FE7C624521
:109B700000D270BDA84214BF4FF080444FF0404463
:109B8000002E08BF0024BEF1806FA8BFA1F1C04124
:109B9000BDE8704080F282804FF0000001F1C041CA
:109BA00001F0004170479EEA0C0F0CEA131518BF34
:109BB00095EA0C0F06D04FF0000081EA030E0EF07C
:109BC000004170BD00F01CF88900013E00F007B8AC
:109BD00000F009B84FEA430C5FEA5C5C08D081EA08
:109BE000030100F05BB84FEA410C5FEA5C5CF6D120
:109BF0004FF00000014970470000FF070000F87FA8
:109C00000EF1020E2EF0030E5EF8046B364205D400
:109C1000012A43EB030515F5001F12D8012841EB7B
:109C2000010C1CF5001F0CD80ED14FEAD17C15F5A4
:109C3000001F0CEB4C0C0CF1020C08BF4CEBD37C5E
:109C400004E04FF0080C01E04FEAD37C0CEB4C052C
:109C500026FA05F606F00706B6F1040C06D20EEB5E
:109C6000860CBDE870404CF0010C6047DFE80CF05A
:109C7000090B02024FF000414FF00000A1F5002156
:109C800070BD19461046012851EB010418BFD4F5E8
:109C9000001484BF002001F0004170BD0808A0F549
:109CA00000114FEA31017047F7F748BAF7F77CBB6C
:109CB000000000000000000001020304060708097C
:109CC00000000000010203040000000024F1501213
:109CD00034563134646F670000000000400100001A
:109CE000000600001C4D0020010A0000224D00204B
:109CF000020400002C4D0020303132333435363729
:109D000038394142434445464030580030313233BF
:109D100034353637383961626364656640307800BF
:109D20000400000800000000000000020001000024
:109D3000100000000000000000000000303132334D
:109D4000343536373839616263646566787000305F
:109D50003132333435363738394142434445465839
:109D60005000000002400000000000A000000000C1
:109D700005400000000000C8000000000C4000008A
:109D80000000409C00000000194000000020BCBE04
:109D90000000000034400000BFC91B8E000000041A
:109DA000B5400000504BCFD06607E2CF0100000065
:109DB0006C4100003E8251AADFEEA7340100000092
:109DC000D9420000DCB5A0E23A301F97FFFFFFFF49
:109DD000B4450000FD25A0C8E9A3C14FFFFFFFFF68
:109DE000FF3F00000000008000000000FF3F000077
:109DF000000000800000000063616E5F6572726F9A
:109E0000722C636F64653A307825782C2052454374
:109E10003A25642C205445433A25642C204C454374
:109E20003A307825782C20455747463A25642C202F
:109E3000455056463A25642C20424F46463A256402
:109E400000000000909F0008000000204C28000047
:109E50006C0100088CA200084C2800201C3E000069
:109E6000C80100081001000043000000F8FFFFFFD8
:109E7000004040404040404040404141414141401D
:109E800040404040404040404040404040404040D2
:109E90004005020202020202020202020202020261
:109EA0000220202020202020202020020202020266
:109EB00002029090909090901010101010101010BE
:109EC00010101010101010101010101002020202CA
:109ED000020288888888888808080808080808080E
:109EE000080808080808080808080808020202020A
:109EF0004000000000000000000000000000000022
:109F00000000000000000000000000000000000051
:109F10000000000000000000000000000000000041
:109F20000000000000000000000000000000000031
:109F30000000000000000000000000000000000021
:109F40000000000000000000000000000000000011
:109F50000000000000000000000000000000000001
:109F600000000000000000000000000000000000F1
:109F7000000000001C00000043000000F8FFFFFF8D
:109F80000C0000000E0000000F0000002E0000007A
:109F9000915324F432100235018D010612DF3B1279
:109FA0000D1422F101000AFF01020304050607084F
:109FB0000901FA03FF600401FF01FF01FF01FF0136
:109FC000FF012413219102140813D1901408C182B7
:109FD000140811972408030F04FFF4010301FF0183
:109FE000A303FF600401FF01FF01FF01FF01FF0167
:109FF0002413219102140813D1901408C18214086B
:10A0000011972408030F04FFF4010301FF01A303C8
:10A01000FF600401FF01FF01FF01FF01FF012413A5
:10A02000219102140813D1901408C18214081197C9
:10A030002408030F04FFF4010301FF01A303FF60E1
:10A040000401FF01FF01FF01FF01FF012413219122
:10A0500002140813D1901408C1821408119724081F
:10A06000030F04FFF4010301FF01A31AFF011360B2
:10A07000022A20084B4C0B084B38140813241D826D
:10A0800020E30104521300FF00891112239B3224A4
:10A0900046AD573665BF74488CC19D5AAFD3BE6C70
:10A0A000CAE5DB7EE9F7F88110080193331A22A58F
:10A0B000562C47B7753E64C99C408DDBBF52AEED50
:10A0C000DA64CBFFF976E802218B3010029913266F
:10A0D00067AF763444BD554AADC3BC588ED19F6E30
:10A0E000EBE7FA7CC8F5D983310A2091121803A74F
:10A0F000772E66B5543C45CBBD42ACD99E508FEF10
:10A10000FB66EAFDD874C904428D5316619F702026
:10A1100004A9153227BB364CCEC5DF5EEDD7FC68EF
:10A1200088E1997AABF3BA85520C4397711E60A10E
:10A13000142805B3373A26CDDE44CFDFFD56ECE9CF
:10A14000986089FBBB72AA06638F7214409D5122EE
:10A1500025AB343006B9174EEFC7FE5CCCD5DD6AAF
:10A16000A9E3B8788AF19B87730E6295501C41A3CE
:10A17000352A24B1163807CFFF46EEDDDC54CDEB8F
:10A18000B962A8F99A708B1023088481951AA79355
:10A19000B62CC2A5D33EE1B7F04008C919522BDB5B
:10A1A0003A644EED5F766DFF7C899400DE00859BFE
:10A1B000B712A6ADD224C3BFF136E0C1184809D307
:10A1C0003B5A2AE55E6C4FF77D7E6C0AA583B41876
:10A1D0008691972EE3A7F23CC0B5D14229CB3850E7
:10A1E0000AD91B666FEF7E744CFD5D8BB502A49996
:10A1F000961087AFF326E2BDD034C1C3394A28D1C7
:10A200001A580BE77F6E6EF55C7C4D0CC685D71E29
:10A21000E597F42880A1913AA3B3B2444ACD5B56A6
:10A2200069DF78600CE91D722FFB3E8DD604C79F55
:10A23000F516E4A9902081BBB332A2C55A4C4BD786
:10A24000795E68E11C680DF33F7A2E0EE787F61CF5
:10A25000C495D52AA1A3B03882B193466BCF7A5466
:10A2600048DD59622DEB3C700EF91F8FF706E69D15
:10A27000D414C5ABB122A0B9923083C77B4E6AD546
:0CA28000585C49E33D6A2CF11E780F0089
:0400000508000131BD
:00000001FF
